:10000000601D00206D3F0000298A0000413F000074
:10001000413F0000413F0000413F00000000000060
:10002000000000000000000000000000453C00004F
:10003000413F000000000000ED3B0000413F000098
:10004000F93C0000F93C0000F93C0000F93C0000DC
:10005000F93C0000F93C0000F93C0000F93C0000CC
:10006000F93C0000F93C0000F93C0000F93C0000BC
:10007000F93C0000F93C0000F93C0000F93C0000AC
:10008000F93C0000F93C0000F93C0000F93C00009C
:10009000F93C0000F93C0000F93C0000F93C00008C
:1000A000F93C0000F93C0000F93C0000F93C00007C
:1000B000F93C0000F93C0000F93C0000F93C00006C
:1000C000F93C0000F93C0000F93C0000F93C00005C
:0C00D000F93C0000F93C0000F93C000085
:1000DC0053B94AB9002908BF00281CBF4FF0FF31A3
:1000EC004FF0FF3000F00CB8ADF1080C6DE904CE08
:1000FC0000F008F8DDF804E0DDE9022304B07047F5
:10010C00704700BF2DE9F04F07468C460846099E04
:10011C0015463C461946002B40F0C6808242B2FA86
:10012C0082F746D94FB1C7F1200E24FA0EFE00FA21
:10013C0007F3BD404EEA030CBC404FEA15481FFACA
:10014C0085FEBCFBF8F9220C08FB19C309FB0EFA5F
:10015C0042EA03439A4528D9EB1809F1FF3004D23F
:10016C009A4502D9A9F102002B44A3EB0A03A4B2CD
:10017C00B3FBF8F208FB123302FB0EFE44EA034415
:10018C00A64514D92C1902F1FF3303D2A64501D987
:10019C00931E2C44A4EB0E0443EA00401EB1FC4019
:1001AC00002334607360BDE8F08F4846DDE71346EA
:1001BC00F0E702B9FFDE87BB831A01214FEA154E27
:1001CC00AAB2B3FBFEFC200C0EFB1C330CFB02F89A
:1001DC0040EA0343984563D9EB180CF1FF3004D285
:1001EC00984502D9ACF102002B44A3EB0803A4B24E
:1001FC00B3FBFEFC0EFB1C330CFB02F244EA034483
:10020C00A2424FD92C190CF1FF3304D2A24202D9CD
:10021C00ACF102032C44A41ABEE7C7F1200C20FA5F
:10022C000CF800FA07F324FA0CFCBD404CEA03026C
:10023C004FEA154EABB2B8FBFEFC110C0EFB1C804A
:10024C000CFB03F941EA0040814504FA07F423D979
:10025C0028180CF1FF3104D2814502D9ACF102010E
:10026C002844A0EB090092B2B0FBFEFC0EFB1C0074
:10027C000CFB03F842EA004398450FD9EB180CF13C
:10028C00FF3204D2984502D9ACF102022B44A3EB05
:10029C00080342EA014191E76146E2E76246F6E76C
:1002AC006046A2E76346B6E7834205D90EB1C6E9BC
:1002BC0000700021084676E7B3FA83F181B98342D6
:1002CC0001D3BA420AD8BC1A60EB030301209C4646
:1002DC00002E68D0C6E9004C002164E70846F7E719
:1002EC00C1F1200C8B4022FA0CF41C4302FA01F5EC
:1002FC0000FA01F327FA0CF220FA0CFB4FEA14492E
:10030C001343BBFBF9F81FFA84FE09FB18BB1A0C4C
:10031C0008FB0EFA42EA0B42924507FA01F73ED966
:10032C00A21808F1FF3004D2924502D9A8F10200BC
:10033C002244A2EB0A029BB2B2FBF9F809FB182289
:10034C0008FB0EFE43EA024296452AD9A21808F190
:10035C00FF3304D2964502D9A8F10203224443EAA2
:10036C000040A0FB0593A2EB0E029A42CE469846A3
:10037C0002D306D14F4504D2B9EB050E63EB04084A
:10038C00013886B1B7EB0E0362EB080707FA0CFCD9
:10039C00CB404CEA0303CF40C6E900379CE740460C
:1003AC00C7E74346DBE73146FDE600001FB51448BE
:1003BC0006F0FDFF002004F02BF928B9114805B018
:1003CC005DF804EB06F0F3BF002301930393694639
:1003DC000123029307F05AF8011E05DA0A4806F0C9
:1003EC00E6FF05B05DF804FB029B9B07FCD103996B
:1003FC0009B10648F3E7064806F0D9FFF1E700BF5C
:10040C00E8A5000005A6000026A6000040A60000F6
:10041C0060A6000008B5054B04225A700821044B55
:10042C00044A07F0C3FC002008BD00BF00000020F8
:10043C0073A600008CA6000008B5054B03225A7069
:10044C000821044B044A07F0B1FC002008BD00BF92
:10045C00000000209BA600008CA6000008B5054BF0
:10046C0002225A700821044B044A07F09FFC00201A
:10047C0008BD00BF00000020B4A600008CA6000040
:10048C0008B5054B01225A700821044B044A07F0A9
:10049C008DFC002008BD00BF00000020CFA600008E
:1004AC008CA6000010B5054B054A00245C70082191
:1004BC00044B07F07BFC204610BD00BF0000002061
:1004CC008CA60000E8A60000034BD8229A700821E5
:1004DC00024B034A07F06ABC0000002001A7000091
:1004EC0020A70000034BFF229A700821024B034AFD
:1004FC0007F05CBC000000202EA7000020A7000025
:10050C00034BEC229A700821024B034A07F04EBCB5
:10051C00000000204DA7000020A70000034BF02294
:10052C009A700821024B034A07F040BC00000020DF
:10053C006CA7000020A70000034BF4229A7008213E
:10054C00024B034A07F032BC000000208BA70000CE
:10055C0020A70000034BF8229A700821024B034A93
:10056C0007F024BC00000020AAA7000020A7000070
:10057C00034BFC229A700821024B034A07F016BC6D
:10058C0000000020C8A7000020A70000034B002299
:10059C009A700821024B034A07F008BC00000020A7
:1005AC00E6A7000020A70000034B03229A70082145
:1005BC00024B034A07F0FABB0000002001A8000020
:1005CC0020A70000034B04229A700821024B034A17
:1005DC0007F0ECBB000000201FA8000020A70000C3
:1005EC0008B5054B02221A700821044B044A07F087
:1005FC00DDFB002008BD00BF000000203DA800006E
:10060C0057A8000008B5054B01221A700821044BAD
:10061C00044A07F0CBFB002008BD00BF00000020FF
:10062C0071A8000057A8000010B5054B054A00241E
:10063C001C700821044B07F0B9FB204610BD00BF0D
:10064C000000002057A800008BA8000030B5374DE3
:10065C00374A85B00821044607F0A8FB6B78042BB9
:10066C001FD8DFE803F01618031A1C00314B324A6E
:10067C000821204607F09AFBAB78EC2B4DD016D80E
:10068C00042B21D00FD8002B41D0032B3DD02B4A6B
:10069C001CE02B4BEBE72B4BE9E72B4BE7E72B4B0A
:1006AC00E5E72B4AE4E7D82BF1D12A4B0DE0F82BE8
:1006BC002FD005D8F02B2ED0F42BE8D1264B04E00C
:1006CC00FC2BE4D1254B00E0254B264A0821204683
:1006DC0007F06CFB2B78012B21D0022B21D013BB04
:1006EC00214B224A2046082107F060FBEB6802935D
:1006FC00AB6801932B7900932046EB781C4A0821B8
:10070C0007F054FB002005B030BD1A4BDDE71A4B47
:10071C00DBE71A4BD9E71A4BD7E71A4BD5E71A4B3D
:10072C00DFE71A4BDDE71A4ADCE700BF00000020C8
:10073C00A3A80000B4A600008CA60000D7A8000057
:10074C00E8A60000CFA600009BA6000073A6000040
:10075C00B0A8000001A700008BA70000C8A70000EC
:10076C001FA8000020A700008BA8000057A80000BD
:10077C000FA9000001A80000E6A70000AAA700002E
:10078C006CA700004DA7000071A800003DA8000058
:10079C00EDA80000012938B505460C4603D107F039
:1007AC002AFB204638BD022907D913680D4A0121BE
:1007BC0007F0FCFA6FF01500F4E7506808F035F913
:1007CC005028034605D9084A0121284607F0EEFABD
:1007DC00F0E7064A0821D0702846054A07F0E6FAE9
:1007EC000020DFE76AA9000084A9000000000020B7
:1007FC00A6A90000012938B505460C4603D107F01F
:10080C00FAFA204638BD022907D913680D4A01218E
:10081C0007F0CCFA6FF01500F4E7506808F005F912
:10082C005028034605D9084A0121284607F0BEFA8C
:10083C00F0E7064A082110712846054A07F0B6FA77
:10084C000020DFE76AA9000084A900000000002056
:10085C00C0A90000012938B505460C4603D107F0A4
:10086C00CAFA204638BD022907D913680D4A01215E
:10087C0007F09CFA6FF01500F4E7506808F0D5F813
:10088C006328034605D9084A0121284607F08EFA49
:10089C00F0E7064A082190602846054A07F086FAD8
:1008AC000020DFE76AA90000D8A9000000000020A2
:1008BC0000AA000070B50F4C237805461BB100F060
:1008CC000FFC002323700C4C00211022204608F052
:1008DC0067FA0A4B5A785B88A38000262046627020
:1008EC00267000F045FB2846054A082107F05EFA01
:1008FC00304670BDD20A0020B80500200000002050
:10090C0017AA0000F8B51C4C237805460F4616466E
:10091C001BB100F0E5FB00232370022F08D92846F9
:10092C003368164A012107F041FA6FF01500F8BD43
:10093C00134C10220021204608F032FA01232370B8
:10094C00104B5A7862709A782271022FDA781B78E1
:10095C00A271637105D1706808F067F80A4BA0604A
:10096C00E360074800F004FB2846084A082107F01A
:10097C001DFA0020DBE700BFD20A00202DAA0000E0
:10098C00B805002000000020090B000048AA000058
:10099C00012938B505460C4603D107F02CFA204640
:1009AC0038BD022907D91368164A012107F0FEF950
:1009BC006FF01500F4E7506808F037F85A2805D99D
:1009CC00114A0121284607F0F1F9F1E70F4C104DBF
:1009DC001022E8600021204608F0E2F9052323707C
:1009EC006B786370AB7823712B786371EB78A371A0
:1009FC002046EB68A36000F0BBFA064B01221A708C
:100A0C000020CDE72DAA000068AA0000B805002040
:100A1C0000000020D20A002038B50F4C05460021FA
:100A2C001022204608F0BCF9042323700B4B5A7893
:100A3C006270DA78227120461A799B686271A36021
:100A4C0000F096FA064B01221A702846054A082136
:100A5C0007F0ACF9002038BDB805002000000020DC
:100A6C00D20A00208EAA000038B50F4C0546102281
:100A7C000021204608F094F9032323700B4B5A787D
:100A8C009968627020461A795B88A160A380A27174
:100A9C0000F06EFA064B01221A702846054A08210E
:100AAC0007F084F9002038BDB805002000000020B4
:100ABC00D20A002098AA000010B50D4C23781BB167
:100ACC0000F00EFB002323700A4C0021102220465C
:100ADC0008F066F902232370074B5A78627020469F
:100AEC00DA781B786271237100F042FA002010BD95
:100AFC00D20A0020B805002000000020014806F0B2
:100B0C0056BC00BFA2AA00001FB504460C2200214F
:100B1C0001A808F045F901A800F0ECFA2046094AB2
:100B2C00082107F043F9DDE90112204607F04BF9E3
:100B3C002046039B044A082107F038F9002004B032
:100B4C0010BD00BFC1AA0000D4AA0000012938B50D
:100B5C0005460C4603D107F04EF9204638BD022954
:100B6C0007D91368104A012107F020F96FF015001E
:100B7C00F4E7506807F059FF012805D90B4A012109
:100B8C00284607F013F9F1E7C0B206F0D4FB4FF09A
:100B9C0080432846D3F87835054A03F00103082131
:100BAC0007F004F90020D9E76AA90000EBAA0000BD
:100BBC0008AB0000014800F0ABBA00BFB80500203C
:100BCC00012910B50C4603D107F015F9204610BDCC
:100BDC00022907D91368064A012107F0E7F86FF0DC
:100BEC001500F4E702D15368024AF5E70020EEE75E
:100BFC002DAA000032AB0000012910B50C4603D120
:100C0C0007F0F9F8204610BD022907D91368064AE7
:100C1C00012107F0CBF86FF01500F4E702D153680F
:100C2C00024AF5E70020EEE72DAA000047AB0000D2
:100C3C00012910B50C4603D107F0DDF8204610BD94
:100C4C00022907D91368064A012107F0AFF86FF0A3
:100C5C001500F4E702D15368024AF5E70020EEE7ED
:100C6C006AA9000032AB00000B4B00224FF0FF31A1
:100C7C00C3F80022C3F80813C3F81021D3F81021CD
:100C8C0001221A61D3F81021002AFBD00022C3F8EC
:100C9C001021D3F81031704700100040114BD3F8DD
:100CAC00302110B542B110490022C3F83021D3F8DD
:100CBC0030210A6801320A60D3F80C218AB1002273
:100CCC00C3F80C21094AD3F80C31136801331360B3
:100CDC008268934205D1FFF7C7FFBDE81040C36897
:100CEC00184710BD00100040C8050020CC0500209E
:100CFC0073B5194B194E187030460C4605F058F860
:100D0C00174B0021D3F80022C3F800124FF0FF322A
:100D1C00C3F80823D3F810554FF47A52A4FB0243BE
:100D2C00EAB2C2F1200503FA05F5A2F1200024FA7B
:100D3C0002F223FA00F02A430123024300933046C7
:100D4C0008F0D0FB304608F0B3FB304602B0BDE8EB
:100D5C00704005F01FB800BFD30A002084A000002B
:100D6C00008000401FB52D4B40F20122C3F85026E5
:100D7C000022C3F83425C3F83825C3F82C250122EA
:100D8C0091420446C3F8302542D002293AD00029BA
:100D9C0036D1AB22C3F824254FF0AB320021C3F877
:100DAC001C2501A80A2207F0FBFF042C0CBF012212
:100DBC0000221B4B0BBF8DF808208DF8082040F249
:100DCC0007124FF483721A809DF806309DF80520A7
:100DDC001B0443EA02239DF80720002A18BF4FF496
:100DEC0080119DF8082008BF00210B4343EA0263E1
:100DFC000A4A43F00803C2F814350A4BC2F81835F6
:100E0C0004B010BDCC22C3F824254FF0CC32C5E77A
:100E1C006A22C3F82425044AC0E700BF0010004032
:100E2C00D00A0020FF0004031B81FE5870B50C464D
:100E3C00FFF798FF114A1249FF231370F02000238B
:100E4C00CC250133DBB284B9C1F80041D1F8006183
:100E5C00D1F80061002EFBD0D1F80865D654FF2BD9
:100E6C00EFD1084BC3F8042570BD022C01D1D55429
:100E7C00F5E7012C08BFD054F1E700BFD40B0020DC
:100E8C0000D0004000100040014BC3F8080570472B
:100E9C0000100040F8B5104C16460D46FFF7E4FE66
:100EAC00C4F81005D4F8003243F02103C4F8003222
:100EBC000A4BC4F804353146FFF754FF2846FFF7B8
:100ECC00E3FF074B00221A604FF48053C4F804333D
:100EDC0001236360F8BD00BF00100040D40A00205D
:100EEC00C8050020B0F5A07F70B50C4632D109784A
:100EFC0003291FD11B4B667818782579FFF7B4FEB0
:100F0C00194AC2F81065D2F8003243F00103C2F856
:100F1C000032C2F80C55FFF7B7FF0123136062795A
:100F2C00A07910490B780133DBB2834298BF1A4683
:100F3C000A7070BD042908D10A4B2279607819789F
:100F4C00FFF7A8FF22796079EBE7BDE8704007480E
:100F5C0006F02DBAB0F5A27F02BF034B01221A6036
:100F6C00E7E700BFD30A00200010004071B1000079
:100F7C00F7B502780346052A18D8DFE802F0031902
:100F8C00424A5154457804794079FFF76DFE4E4A38
:100F9C00C2F81055D2F8003243F00103C2F8003207
:100FAC00C2F80C45FFF770FF0123136003B0F0BDCE
:100FBC004478067985794079FFF756FE014620463C
:100FCC00FFF734FF404A4149D2F8003243F0210385
:100FDC00C2F800322846C2F81045C2F80C65FFF77B
:100FEC0053FF00230B60C2F80C31D2F80C310823EC
:100FFC00C2F8043301231360D2F80C31002BFBD060
:10100C00D4E702794179407803B0BDE8F040FFF7AE
:10101C0041BF8168407903B0BDE8F040FFF768BE7E
:10102C0081680079F7E745780779847940799E687B
:10103C00FFF71AFE01462846FFF7F8FE224BC3F8CD
:10104C001055D3F8001241F00301C3F800122046EA
:10105C00C3F80C75FFF718FF1D4B1E485A5D1E4B4D
:10106C001C886243C6F164045443B4FBF6F4144484
:10107C0004F09EFE194BD3F800220022C3F8002284
:10108C004FF0FF32C3F80823D3F81025D2B2210F4A
:10109C00C2F12003240101FA03F3A2F1200024FA87
:1010AC0002F221FA00F01A430121024300910223BB
:1010BC00084808F017FA074808F0FAF9054803B091
:1010CC00BDE8F04004F066BE00100040CC050020E6
:1010DC00ACB1000084A00000D00A002000800040C9
:1010EC0008B5034804F064FEBDE80840FFF7BCBD3A
:1010FC0084A00000044B03604FF480734360034BE7
:10110C001B688360704700BFD40A0020C80500200C
:10111C0030B5134B01221A60124B134A85B0CDE93E
:10112C00023002A90446114804F0E6FD104B984227
:10113C00014602D00F4806F03AF90025002206219C
:10114C00082007F056FC0C4A009523460621012086
:10115C0007F057FC012002F0E9FC284605B030BD31
:10116C0000D0004004000200F10E000084A000003A
:10117C000000AD0B8BB10000A90C00000B68013313
:10118C000B60014B1B68184710000020014B1860C6
:10119C00704700BF1000002007B50B460021024627
:1011AC000191034801A900F0E5F803B05DF804FBD8
:1011BC00891100002DE9F84FB0F8189019F00808C3
:1011CC00044693460DD001290CBF49F0100949F093
:1011DC002009A0F818908BF31188BFF36F8FBDE82E
:1011EC00F88F09F00709022907D1204606F0ECF820
:1011FC000028F0D00128238B4ED16769218B002F5A
:10120C0015DA256821F00701C4E9008841F00101D5
:10121C0021830026218B01F0070ACA4502D0A3685E
:10122C00002B5AD10DB9002E71D0002356E001F0DD
:10123C0007035A1F012A1ED821F00701062B256827
:10124C0089B2C4E900880AD13DB1638B2A46126881
:10125C0001339BB2002AFAD1638341F0020121834E
:10126C00204606F0B1F806460028D3D0238B43F075
:10127C0020032383CDE7042B0CD121F0070189B285
:10128C002183204606F0A0F805460028C1D041F085
:10129C00200121830025BCE7032809D1226923F012
:1012AC000703166843F00603238300252F46B1E796
:1012BC00042806D1226923F00703566843F004037F
:1012CC00F2E7052806D1226923F00703966843F05C
:1012DC000503E9E700252E46E8E7012341F0080164
:1012EC0021838BF31188BFF36F8FFBB985BB16B1CC
:1012FC001F492046B0474FF02003EFF3118B83F3C7
:10130C001288BFF36F8F238B23F008032383238B67
:10131C00DA0625D523F0100323830121B4F81890A5
:10132C0009F0070900297FF45EAF54E7A168002992
:10133C00DCD0D1F80090D1F804B03B4652462046A0
:10134C00D847B9F1000FD1D04946D9F80090F2E74F
:10135C0029463B46524620462D6806F051F8C5E713
:10136C0013F020011EBF23F0200323830221D5E7B5
:10137C00397400002DE9F04F91B08B4602909246E3
:10138C001C4600259AF8000008B928465FE325287A
:10139C000AF1010707D0029B594698470028C0F272
:1013AC005683013512E2182200210AA807F0F8FC36
:1013BC009AF80130252B78D0002210469646944698
:1013CC001646394617F8013B2B2B00F09D8000F296
:1013DC009480202B00F09B80232B00F09B802EB15F
:1013EC009DF8306046F004068DF83060BCF1000FBB
:1013FC0005D09DF8306046F008068DF83060BEF1DF
:10140C00000F05D09DF8306046F010068DF8306066
:10141C0028B19DF8300040F020008DF830002AB142
:10142C009DF8302042F040028DF830209DF830209D
:10143C0002F04400442803D16FF386128DF830205B
:10144C009DF830202A2B42F080028DF830207BD181
:10145C009DF8312042F001024B1C8DF831201A7896
:10146C002E2A9DF831200CBF0121002161F341028D
:10147C008DF8312074D15A782A2A6AD00133002190
:10148C000A26184610F8012BA2F13007092F40F25A
:10149C008E809DF830200E91C2F3400040EAD1714D
:1014AC0061F341028DF830205AE00AF102078DF801
:1014BC0033309DF83130D90740F1498154F8049B01
:1014CC00B9F1000F07DA9DF8302042F004028DF8D4
:1014DC003020C9F100095A0740F1428154F8048BBD
:1014EC00B8F1000F80F241819DF831306FF3410368
:1014FC008DF831304FF0FF3837E12D2B0CD0302BDD
:10150C007FF46DAF01225CE74FF0010C59E74FF00F
:10151C00010E56E7012054E7012652E70CFB0202AC
:10152C00303A33461E4616F8010BA0F13007092F4E
:10153C00F4D9994293D09DF830100D92D20F62F3EA
:10154C0041018DF830108AE70B4600224FF00A0C4F
:10155C00E8E79DF8312042F004028DF83120023387
:10156C001F4617F8012B6C2A41D025D8682A2BD09E
:10157C006A2A46D04C2A4CD01F4617F8012B9DF8EE
:10158C0031308DF83320782A00F2D980572A4DD883
:10159C00412A03D0453A022A00F2D1809DF832301C
:1015AC00042262F302038DF8323001239EE006FB25
:1015BC0001213039034664E7742A26D07A2ADBD11C
:1015CC009DF8313006220DE05A78682A9DF83120BA
:1015DC0006D1012161F3C6028DF831209F1CCCE7A6
:1015EC001346022262F3C6038DF83130C5E75A78F0
:1015FC006C2A9DF8312001D10421EBE7134603221C
:10160C00F0E79DF831300522ECE79DF831300722E8
:10161C00E8E7BDF8303023F4F04323F0020343F441
:10162C00804343F00203ADF83030A6E7A2F1580135
:10163C00202900F2848001A050F821F00D17000041
:10164C004B1700004B1700004B1700004B17000006
:10165C004B1700004B1700004B1700004B170000F6
:10166C00A91500004B1700000D170000CD16000047
:10167C00A9150000A9150000A91500004B170000C2
:10168C00CD1600004B1700004B1700004B17000045
:10169C004B170000151700000D1700003117000044
:1016AC004B1700004B170000311700004B170000C0
:1016BC000D1700004B1700004B1700000D17000012
:1016CC009DF83210012003F0780360F30201402BE7
:1016DC008DF8321002BF9DF8301041F001018DF8E9
:1016EC003010632A31D1003B18BF01239DF8302004
:1016FC00C2F340010B4363F341028DF83020D8E66E
:10170C009DF832100220DEE79DF8322003F07803BA
:10171C00A3F14000032161F3020243428DF8322011
:10172C004341E3E79DF83220032113F0780F61F376
:10173C0002028DF8322014BF01230023D6E79DF856
:10174C00303043F001038DF830300023CEE79DF9A3
:10175C003020002AB4BFDDF834904FF0FF39BAE6E0
:10176C009B077FF5C7AEDDF838809DF8311000235C
:10177C00CDE90D339DF8323003F00703012BC1F393
:10178C00C30138D1CB1E042B22D8DFE803F00309A8
:10179C000921210054F8043BDA17CDE90A3206E09E
:1017AC00073424F00704F4E80223CDE90A239DF85A
:1017BC00303013F0030656D002983B465246594639
:1017CC0005F062FF0028C0F242810544BA46D9E513
:1017DC0054F8043B01294FEAE372CDE90A3205D1F2
:1017EC009DF828300A9300230B93E0E70229DED101
:1017FC00BDF92830D0E7022B23D1CB1E042B13D8F4
:10180C00DFE803F0030A0A12120022680A9200238E
:10181C00201D0B930446CAE7E01D20F00700F0E8FA
:10182C000223CDE90A23F5E754F8043B0A93012976
:10183C004FF000030B93D3D00229B8D1BDF8283058
:10184C00D0E7042B09D1E31D23F0070303F10804AF
:10185C00D3E90023CDE90A23A9E7032B04BF54F8ED
:10186C00043B0A93A3E79DF833007828AED862288E
:10187C0022D825283FF48FAD5828A7D10DF1260387
:10188C000093DDE90A0104AB0CAA05F0B7FE824611
:10189C00B8F1000F0DF126000CDB9DF83020A0EB09
:1018AC000A036FF3861298458DF8302002D9A8EB05
:1018BC0003030D9380463DE06338152886D801A2BA
:1018CC0052F820F051190000B5190000D91700008A
:1018DC00D9170000D9170000D9170000B51900005E
:1018EC00D9170000D9170000D9170000D91700002C
:1018FC000F1A0000DD190000E1190000D9170000D3
:10190C00D917000029190000D9170000DD190000B3
:10191C00D9170000D9170000DD190000B8F1000F2D
:10192C00DDF828A00ADB4146504607F0DFF90AEB48
:10193C0000080026BAF1000F0CD147E7504607F01B
:10194C00CEF9F4E70A9B8DF8103000260DF1100A41
:10195C000DF11108A8EB0A0306B101339DF83220F2
:10196C00D00668D5023352060D9948BF0E9A0B4427
:10197C0048BF9B18B9F1000F76DD9DF83020A9EB1C
:10198C000309C2F38003039353076DD4500661D54A
:10199C0046B1029B594630469847002857DB039BBB
:1019AC0001351E46302356E01E070FD413F01006E7
:1019BC0018BF2026DDE90A23002BBFF65FAF524289
:1019CC0063EB4303CDE90A232D2657E72B26F1E7DA
:1019DC00002653E70A9840B30DF1260300930CAA96
:1019EC0004AB002105F00AFEBDF8323003F0EF0322
:1019FC0043F4F04343F010038246ADF83230002636
:101A0C0046E70A9B07293FF6E1AEDFE801F00C043C
:101A1C00060C08080C0C1D70D8E61D80D6E6EA17DB
:101A2C00C3E90052D2E61D60D0E6DFF8C8A0064636
:101A3C000AF105088EE7110748BF013393E71846F2
:101A4C0003935946029B98470028039B04DA11B074
:101A5C00BDE8F08F20234D444A46002AA5EB09012E
:101A6C0009F1FF39EBDC0D4636B1029B5946304685
:101A7C0098470028EBDB01359DF83230D90601D4AC
:101A8C001A0706D5029B5946302098470028DEDB02
:101A9C0001359DF83230DB0607D59DF83300029BEB
:101AAC00594698470028D2DB01350D9E2E44731BF6
:101ABC00002B16DC029843465246594605F0E4FDCD
:101ACC000028C4DB0544A944A9EB0503002B7FF7D0
:101ADC007DAE029B5946202098470028B7DB013584
:101AEC00F2E7029B5946302098470028AFDB0135BE
:101AFC00DDE700BFBCB1000008B54FF02002EFF3EA
:101B0C00118382F31288BFF36F8F02F0B3FB03488B
:101B1C0005F04DFC01F0DEFFFCE700BFC2B1000098
:101B2C0013B5044604F04CFCC0F307230193C0F337
:101B3C0007430093044A030E0821204606F036F9A9
:101B4C00002002B010BD00BFEBB1000010B5044680
:101B5C0007F078FE4FF47A73A0FB032003FB01031C
:101B6C00D20B42EA43432046024A082106F01EF9F2
:101B7C00002010BD04B2000010B5044603F0F4FAC6
:101B8C00084A03460821204606F010F9064A20466A
:101B9C00082106F00BF90548214604F09FFA0020B5
:101BAC0010BD00BF13B2000032B20000BD1B00001C
:101BBC00F0B587B0D0F8A07004460D4607F0F6FCDF
:101BCC00064605F019F8234B234A002E08BF1E4683
:101BDC00224BCDE90046844218BF13460821284603
:101BEC001F4A06F0E3F8D4E90A23CDE9022394F95D
:101BFC000E301C4A00930821237B284606F0D6F8A9
:101C0C00204604F0B3FA626E00920346164A08218D
:101C1C00284606F0CBF805A9204607F0D7FC03466A
:101C2C0030B1124A0821284606F0C0F807B0F0BDC2
:101C3C00059A6423B91ACDE900214B430C4AB3FB36
:101C4C00F7F30821CDE9027328463B4606F0AEF8BF
:101C5C00ECE700BF3EB200008BB900003CB20000C4
:101C6C0041B200004DB2000079B2000090B2000009
:101C7C00BDB2000070B5134E88B004460146124840
:101C8C0004F02CFA07AA4FF40061304607F092FCDE
:101C9C0007996422C1F5006042434FF400630025AC
:101CAC00D20ACDE90303CDE9013105922046074A5A
:101CBC000095A6F12003082106F078F8284608B014
:101CCC0070BD00BF001F0020F91C0000F4B2000022
:101CDC0010B5044607F0E8FA034A034608212046EB
:101CEC0006F064F8002010BD3AB30000F0B5D0F84F
:101CFC00A06089B004460D4607A907F067FC0346AF
:101D0C0030B1104A0821284606F050F809B0F0BD51
:101D1C00204607F04BFC07990B4A771A002818BF8E
:101D2C0002466423CDE90217CDE900267B43074A1E
:101D3C00B3FBF6F30821CDE904632846234606F0ED
:101D4C0035F8E3E790B200003EB2000050B300005B
:101D5C000346006810B50C46114608B1027822B94A
:101D6C00024A204602F056FA204610BD5AB4000032
:101D7C0010B50C68D1E90112FFF7EAFF034A0346DC
:101D8C000821204606F012F8002010BD5FB40000B8
:101D9C002DE9F0478AB0054601A804F0BFF8019E72
:101DAC001B4ADFF87080DFF87090DFF870A0182302
:101DBC0003FB00660821284605F0F8FF019CB4429D
:101DCC0003D300200AB0BDE8F08705AF39461422D2
:101DDC002046FFF7BDFF424603460821284605F082
:101DEC00E5FF204607F09BFB0D4A002814BF4B462D
:101DFC0053460821284605F0D9FF142320460949EB
:101E0C00049302AACDE90257183407F092FBD6E7E7
:101E1C007EB4000088B400006FB4000075B40000FC
:101E2C008DB400007D1D00002DE9F043114BDFF84F
:101E3C00489053F82140013187B053F82180064671
:101E4C000027A04503D8384607B0BDE8F0832046EC
:101E5C0007F065FB054658B1142201A92046FFF78F
:101E6C0077FF4A4603460821304605F09FFF2F4670
:101E7C001834E6E78CA1000094B4000010B50821DA
:101E8C0004461E4A05F092FF00212046FFF7CCFFC6
:101E9C0020B91B4A0821204605F088FF082120465E
:101EAC00184A05F083FF01212046FFF7BDFF20B93A
:101EBC00134A0821204605F079FF08212046124AD2
:101ECC0005F074FF02212046FFF7AEFF20B90C4A43
:101EDC000821204605F06AFF082120460B4A05F030
:101EEC0065FF03212046FFF79FFF20B9044A082114
:101EFC00204605F05BFF002010BD00BF9AB4000027
:101F0C00A9B40000B1B40000C0B40000CEB400000D
:101F1C008B1E022B2DE9F04107468846144633D818
:101F2C0060681022002106F017FEB8F1020F064679
:101F3C001ED0A0680A22002106F00EFEC5B2214A6E
:101F4C002B460821384605F031FFB8F1040F1ED09E
:101F5C00102D0FD0202D10D0082D10D13378DBB2DE
:101F6C00194A0821384605F021FF0020BDE8F08110
:101F7C002025E4E733889BB2F2E73368F0E7134A95
:101F8C000821384605F012FF6FF01500EEE7E06807
:101F9C001022002106F0E0FD0D4A034604460821FC
:101FAC00384605F003FF102D06D0202D07D0082D44
:101FBC00E5D1E4B23470D8E7A4B23480D5E734600C
:101FCC00D3E700BF32B500005DB5000047B5000097
:101FDC006EB5000070B50E4E044633780D4631B127
:101FEC002BB1BDE870400B4A012105F0DFBE83F038
:101FFC000103337033B1084A0821204605F0D6FEA0
:10200C000123337029462046BDE8704005F008BF17
:10201C00D60C002082B50000BDB5000070B504469A
:10202C003C480378182B02D10B78112B31D0013A94
:10203C000B4655189D4225D18B5C0A780370A2F192
:10204C003003092B344C04D922F02003413B052BDF
:10205C0004D823683149CA54013323602368022B06
:10206C0034D110222D48002106F076FD2C4A13683D
:10207C0003F8010B13602B4A136801331360002320
:10208C00236023E013F8016B182ED3D11E78112E88
:10209C00D0D1244D244A2B680821204605F086FE19
:1020AC0020460021FFF796FF204B187870B9204A84
:1020BC002B681168042B0ADC08B111602B6013F03B
:1020CC0003010BD1126813681BBA136070BD08684A
:1020DC0000BA41F8040B043B0120EBE75B4203F030
:1020EC00030358BF5942022904D1126813885BBA02
:1020FC009BB2EAE70329E9D1106802681104C2F324
:10210C00074301F47F010B4302F47F421343036046
:10211C00DCE700BFD80C0020D4050020D40C002034
:10212C00D0050020DC050020E7B50000D70C00200E
:10213C00D80500202DE9F74F0D462D49DFF8B48066
:10214C00DFF8B490DFF8B4B000230B602C4988F8AA
:10215C00003006460B601446012D274654F8043F08
:10216C0021D9184602224946019306F0D4FD019B61
:10217C0088B922689278003A18BF012203EB020A50
:10218C0020490222504606F0C6FD30B9012388F8DA
:10219C000030013DE0E70022F0E74946504606F0EA
:1021AC00AEFDB0B9043700221146786806F060FC29
:1021BC00154B002211461860786806F059FC134B39
:1021CC00134918603046FFF705FF002003B0BDE847
:1021DC00F08F9AF800202D2AE5D19AF80120002AD8
:1021EC00E1D053465A460821304605F0DFFDD0E7D2
:1021FC00D4050020D70C002001B6000007B6000063
:10220C00DC05002004B60000D0050020D805002015
:10221C002920000013B5094807F081F958B1084A84
:10222C0006491268074800240094012300F064FD5D
:10223C00204602B010BD6FF01200FAE71C9C0000A3
:10224C0028A20000349C000010B50C4611464268D0
:10225C001068C0E90041916883600023C1E9023332
:10226C00C1E905334B600B61D168C1E90233C1E9A7
:10227C0005334B600B61C360A36823B19B6C13B136
:10228C00044920469847A3689B6A0BB1204698479F
:10229C00002010BD3D7B000010B58168044608315C
:1022AC0001F0B0F8A168034A20460831BDE810409F
:1022BC0001F046B8B8B60000014905F0E1BC00BF1A
:1022CC00F2B2000037B504468068D0F864325A0781
:1022DC000D4605D5002105F011FDE06806F098FAD1
:1022EC00E368DB686BB9002D37D0A068423005F08D
:1022FC00C1FCA36898B303F1420103F5A17006F089
:10230C00C4FCA268E0680DF106034232294606F0CF
:10231C0082FA58B9A06800F5A171423006F0B5FCFC
:10232C00A068423005F0A6FCADF80600204606F089
:10233C0048F8A368D3F860329B0603D50949606955
:10234C0005F09EFC204600F0CBFEA368BDF80620ED
:10235C00DA879A87204605F0A1FF03B030BD83F8D9
:10236C004201CEE7409D00002DE9F04F00239FB0C5
:10237C00CDE90533836804464233039306F027F80E
:10238C00204605F077FF10B96069FFF795FFA0684C
:10239C0014220021083006F003FD204605F017FF3B
:1023AC00A168E0688A8F4231002606F06BFA20465D
:1023BC0006F0E9FA4FF0FF38B146B24611AF02967B
:1023CC003546B346DDE90532012A00F0D6800B2BE9
:1023DC0040F2AE80069B022B40F0AE80894B8A4ABD
:1023EC00012114E0039A0223394606A805F083FD67
:1023FC0006997A680392034629B96FF007052846B7
:10240C001FB0BDE8F08F012905D120B17F4A2046CD
:10241C0006F089F8F1E7059B4BB3386801F016F824
:10242C0098B166B1A5680D9608350CAE0FCE0FC5E8
:10243C0033682B602046FFF72FFF0125DFE7744A36
:10244C000121204606F06FF8D7E7059B7BB13A686F
:10245C002946204601F05EF9022800F08E80032800
:10246C0005D0059B0133059301230293AAE7BAF12A
:10247C00000F05D1396807AA584605F027FE054616
:10248C00043708F1FF38002D40D0029AEB6842B1B6
:10249C0013B3204605F09BFF204605F0FFFE5D4A76
:1024AC00CEE7CBB1A368DDF81490AE4603F1080C6F
:1024BC00BEE80F00ACE80F00DEF80030CCF80030BE
:1024CC00AB684BB96B7CFE2B01BF95F8108009F102
:1024DC00010308F1FF380593D5F804C0BCF1000FD7
:1024EC0008D0AE46BEE80F000CAE0FC6DEF80030CA
:1024FC0033606646AB46B8F1000F03D1069B022B46
:10250C007FF460AF059B013305935BE7059B63B9D3
:10251C00A368DB690BB1DB683BB93F4B00933F4AC7
:10252C00119B0121204605F0FEFF4FF0010AE2E766
:10253C00B8F1000F7FF456AF029B4BB1204606F06A
:10254C0043FAA2680C23423211A905A805F0D3FC6A
:10255C00059DA0681EAB03EB8503002243F8342CC9
:10256C00436973B9002E3FF448AFC368B3423FF4DC
:10257C0061AF0D9600F1080557E7059B0B2BDBD9D6
:10258C0028E7037EA5EB0905B3B1417E4FF6FF7238
:10259C00FF2918BF0A469D4202D313449D420BD912
:1025AC0083681F4A0121204605F0BDFF2046FFF736
:1025BC0073FE6FF0150522E74FF4006100F51970FA
:1025CC0005F024FBA06800F53E7005F0B0FBA36895
:1025DC0011AA294602EB89025B69204698470546F9
:1025EC00A0684FF0FF324FF0FF3300F53E7005F05E
:1025FC0054FBA0686FF4006100F5197005F015FB31
:10260C00FDE600BF3BB7000096B40000C6B6000064
:10261C00DAB60000F8B6000027B7000001BA0000D7
:10262C005FB700008368022210B51A719A6B0446DA
:10263C00BAB983F84220DA63D3F86432DB040BD5E1
:10264C000321084B084A05F06EFFA0686FF4805117
:10265C0000F5197005F0E9FA2046BDE8104000F0CD
:10266C0051BE10BD7AB700008AB400002DE9F04FBE
:10267C0004468068ABB0012100F5197005F0C6FA6C
:10268C00A3681B79022B17D100230B93A3686068F6
:10269C009E6B03681D690BABC6B110221DA9A84720
:1026AC000B9A4AB11DA92046B047A3689B6B002B1F
:1026BC00ECD12046FFF7B6FFA0686FF0010100F5E2
:1026CC0019702BB0BDE8F04F05F0AFBA01220DF137
:1026DC002B01A8470B9B002BEED09DF92B209DF8CE
:1026EC002B30A068002AD1DB4279032A00F2FD824C
:1026FC00DFE812F0040075029802FB020D2B1AD0D1
:10270C000A2B18D0B0F864226FF3CA02A0F8642226
:10271C00092B4CD032D8002BB8D0082B00F0C48138
:10272C00A3F120025E2A00F2CB81012105F0E6FA2A
:10273C009DF82B10E8E0D0F86422C2F3C7022AB14E
:10274C00D0F86422C2F3C7029342E1D1B0F86422FC
:10275C00818F63F3CA02A0F8642259B905F0CEFA4E
:10276C00E06806F055F86069FFF7A6FD2046FFF714
:10277C0059FF8BE72046FFF7F7FDF7E71B2B13D02C
:10278C007F2BCDD1D0F860329A077FF57FAF012136
:10279C0005F0B4FAA368D3F860321B0700F18C8102
:1027AC00204605F000FF71E7012343716EE7D0F876
:1027BC0060329E077FF56AAF012105F09FFAA06891
:1027CC00838FFF2B3FF462AFC28F00F1420100F503
:1027DC00A17006F0DAFAA268D38F1344002583F8AF
:1027EC0042511DA90C2302F5A1720DA805F083FB23
:1027FC000D990C293FF64AAF2AAB03EB810343F842
:10280C00345CA368DA8F134493F84130202B00F02A
:10281C006E82093B042B40F26A8201294FD80025B5
:10282C000C950C9B2AAA02EB8303002653F834ACBC
:10283C00504605F01FFAB04681460496374618AA52
:10284C003946284600F0E8FB8346002844D1012E87
:10285C0063D10C9B2AAA02EB830353F8340C05F0CA
:10286C0009FAA268064608324146284600F0D4FB15
:10287C000546006805F0FEF9864206D02968821BE1
:10288C0092B23144204605F08CFEA068C38F0344FD
:10289C0093F84230202B3BD0093B042B38D9D0F88D
:1028AC006032DD072FD5002105F032FA20212046B9
:1028BC0000F0F4FCA068012105F02AFAE6E60139E3
:1028CC0000200EAB009301900CAB1DAA05F01EFC72
:1028DC0005460028A5D1D9E6DBF800004A4651464A
:1028EC0006F019FA68B9DBF8000006F0F8F9049B59
:1028FC00834238BF03469BB2002E08BFB8460493F0
:10290C00013601379BE72021204600F0C7FCBDE6CD
:10291C000121204605F0F5FCB8E67FF6B7AE0C9B1E
:10292C002AAA02EB830353F834AC504605F0A2F903
:10293C00A3680690A3F830B0DFF8D0B20596CDF8B6
:10294C000C80A26803990832284600F065FB039BB3
:10295C00013307460393BAF1000F52D13F68002FA1
:10296C0059D1A2681786059B013B0593E9D1606993
:10297C00FFF7A2FC204600F0C5FC0C9B2AAA02EB38
:10298C00830308F1010953F8340C05F073F941463F
:10299C0013AA0746284600F03FFB8046A068D8F8EB
:1029AC000010FF2200F5A17006F079F9D8F800A00C
:1029BC004FF6FF7818AA4946284609F1010B00F09A
:1029CC002BFB002863D0A368006803F5A1730022D9
:1029DC0013F801CB815C614505D121B101324FF671
:1029EC00FF718A42F4D10FB1BA4208DB424506F1BD
:1029FC00FF36A8BF4246012E1FFA82F847D0D946AF
:102A0C00D8E700680028A9D0069A514606F083F949
:102A1C000028A3D095E7584605F02CF9049BA16833
:102A2C00C21892B24B8D09925846089305F022F9C0
:102A3C000790384605F01EF9099ADDE90713A2EB59
:102A4C000009A068B0F830C0591A91FBF2F292B2AA
:102A5C00BCFBF2F102FB11C20CF1010E92B21FFA97
:102A6C0089F9A0F830E05AB9694A00975B4606210B
:102A7C00204605F058FD4946204600F01BFB72E746
:102A8C00644A3B460621204605F04DFDF3E7B8F1BC
:102A9C00000F3FF4FBADA8EB070292B20AEB070163
:102AAC00204605F07EFDF1E5D0F8603299077FF500
:102ABC00EDAD012105F022F9204605F08FFDE5E58D
:102ACC00D0F8602297077FF5E1AD013B162B3FF65E
:102ADC00DDAD01A252F823F0CD2C0000412B0000FB
:102AEC00492B0000AD270000C12C0000672B000013
:102AFC0099260000992600009926000099260000CE
:102B0C006F2B0000772B000099260000A12B0000F2
:102B1C0099260000AB2B0000992600009926000096
:102B2C009926000099260000AF2B00009926000082
:102B3C00DB2B0000204605F051FCA7E5204605F0F4
:102B4C0046FC204605F096FB10B96069FFF7B4FB14
:102B5C00A068012105F0D2F808E6204605F046FCF5
:102B6C0094E5204605F04BFC90E5D0F860329E06CB
:102B7C0003D52949606905F083F8A368D3F860325E
:102B8C009D0603D52549606905F07AF8204600F0CA
:102B9C00B9FB7BE500212046FFF794FB76E501218C
:102BAC00F9E7204605F00DFCA068002380F84230C0
:102BBC00C363012105F0A2F8A368D3F8603298062C
:102BCC007FF564AD1649606905F05AF85EE520465C
:102BDC0000F0CCFAA068012105F090F856E55B2BCB
:102BEC0001D10223E1E5D0F86022910706D5622BD2
:102BFC0008D14FF0FF31204605F0A7FBA368002257
:102C0C005A7143E5662BF9D10121F4E78AB900002A
:102C1C00BEB700008AB40000459D00004A9D00002C
:102C2C00409D000000224271D0F8602292077FF58F
:102C3C002DAD313B1B2B3FF629AD01A252F823F0F1
:102C4C00C92C0000D52C0000E72C0000BD2C000086
:102C5C00992600009926000099260000992600006C
:102C6C00992600009926000099260000992600005C
:102C7C00992600009926000099260000992600004C
:102C8C00AB2B0000A12B0000672B0000412B000098
:102C9C0099260000C12C000099260000CD2C0000C4
:102CAC00992600009926000099260000D92C0000D6
:102CBC0003234371204605F08AFBE7E403234371A9
:102CCC00204605F07EFBE1E403234371D0F860124B
:102CDC0001F0010181F00101EEE503234371D0F80D
:102CEC0060329B077FF5D2AC5AE500235DE50029E5
:102CFC003FF495ADE4E500BF2DE9F0430446806850
:102D0C008846D0F80C1389B015461F46002961D1AE
:102D1C004FF4447206F044F8A3682268E0681A6025
:102D2C0005F017FEA06800F53E7006F063FC4FF44A
:102D3C002A794FF41A76A068304406F0D5FEA068C4
:102D4C000022831901214844103606F0B0FEB6F576
:102D5C002A7F09F11409EED1A369A068002602218B
:102D6C001E6000F5197004F051FFA3681B4A9A62AB
:102D7C00186804F07FFFA368194A83F82C00606878
:102D8C0066F38205C3F86052036841461D6823460A
:102D9C00A8470546D0B9A36801221A71D4E90901E4
:102DAC0000220023CDE906230E230393109B0495E8
:102DBC00CDE9017300940B4B4FF4006203F078FAE9
:102DCC00A368216AC3F80C0303F0C0F9284609B0C4
:102DDC00BDE8F0836FF07705F8E700BF18005000EE
:102DEC00AB7C0000412E000010B5044680680379CE
:102DFC00012B19D14FF0FF324FF0FF3300F53E702D
:102E0C0004F04BFF0821204600F072F90849606974
:102E1C0004F036FF2046FFF705FCA06800F53E7075
:102E2C0004F085FF002010BD6FF08500FBE700BFAC
:102E3C00F1B20000F8B504464068036800219B68B5
:102E4C00984700283FD12046FFF7CEFF00283AD103
:102E5C001D4F1E4EA06800F52A704FF0FF324FF048
:102E6C00FF33032104F088F80546A0684FF0FF32C9
:102E7C004FF0FF3300F53E7075B104F00EFF2046A5
:102E8C002B46134A012105F04EFBA068BDE8F84023
:102E9C0000F53E7004F04BBF04F0FFFE6068036861
:102EAC005B6903B198473A462046022104F0CCFEF8
:102EBC0020463246002104F0C7FEA06800F53E70A3
:102ECC0004F035FFC6E7F8BDBF7C00007926000092
:102EDC00C4B7000010B50D4A0446082104F066FF83
:102EEC0020460B4A082104F061FF2046094A0821BC
:102EFC0004F05CFF2046084A082104F057FF2046E6
:102F0C00064A002100F01CFA002010BDDBB70000BF
:102F1C0019B8000078B80000CCB8000066B9000001
:102F2C002DE9F04716461F462A4ADFF8AC80DFF839
:102F3C00AC90DFF8ACA00B460821044604F036FF39
:102F4C000025AF4231D9735D4A460821204604F072
:102F5C002DFF0135102D20D1224ADFF88480DFF8B7
:102F6C0088900821204604F021FF0025BD422AD27A
:102F7C00735DA3F120025F2A28BF2E234A46082145
:102F8C00204604F013FF0135102D14D12046174AAA
:102F9C00BDE8F047082104F009BF6A07D1D15246B9
:102FAC000821204604F002FFCBE7424608212046C8
:102FBC0004F0FCFECDE76B07D8D142460821204631
:102FCC0004F0F4FED2E742460821204604F0EEFE5F
:102FDC00D9E700BF7CB9000089B9000083B90000B3
:102FEC008BB900008DB90000AFB900008FB900009B
:102FFC0010B5044613460A4601460648FEF7BAF9D0
:10300C0023691B7923B12046BDE8104004F00BBFA7
:10301C0010BD00BF4B7E000010B50B46144650B9D6
:10302C000E490F4A521AB3EBD20F0FD201EBC30168
:10303C004C68204610BD816841B14A68097839B1A5
:10304C001846214690472368002BF2D10024F0E764
:10305C0014204343D418D358F6E700BF609C0000FB
:10306C00289D00008368D3F860329B0603D5024983
:10307C00406905F0DEB87047509D0000014905F02D
:10308C00D8B800BFF2B200000A1E0DDC0ED04223ED
:10309C008168D1F86012890608D5002A0449406974
:1030AC00B8BF524205F0C5B84123F1E7704700BFE5
:1030BC00ABB900000A1E0DDC0ED044238168D1F898
:1030CC006012890608D5002A04494069B8BF5242EB
:1030DC0005F0AFB84323F1E7704700BFABB9000070
:1030EC00826802494069423205F0A3B88AB40000F4
:1030FC0008290A4616D8836893F82E10914211D0ED
:10310C00082A83F82E20D3F8603205D0990609D509
:10311C000549406905F08DB89B0603D50349406904
:10312C0005F087B8704700BFB2B90000559D00008C
:10313C0038B50D4609780446FFF7DAFF6A78072A96
:10314C0010D8A36893F82F1091420BD083F82F203E
:10315C00D3F860329B0605D560690349BDE8384059
:10316C0005F067B838BD00BFBBB90000F8B583687F
:10317C009A8F0546002A4ED0D88F00284BD041306C
:10318C00184403F142060346C41AB342A4B21946CA
:10319C000DD311F80179202F3BD01946013B08784B
:1031AC00202804D001349E42A4B21946F5D9631CE0
:1031BC004E1C121B1944304605F0CFFDA9688A8FAE
:1031CC00121B92B28A870A440023614282F8423071
:1031DC0009B2284605F095F8AB68D3F860329A0628
:1031EC0003D50D49686905F024F833460B4A0821CC
:1031FC00284605F098F92846FFF734FFAB68D3F85A
:10320C0060329B0607D568690549BDE8F84005F0B2
:10321C0010B80B46B8E7F8BD5A9D00008AB4000000
:10322C005E9D00002DE9F04104460D4617460AB19B
:10323C00FFF718FFA368D3F86022D88F520700F16C
:10324C00420003441FD5184605F049FDDFF84480C1
:10325C00064696B9A3689A8FDA87204604F0F6FFE3
:10326C0020B107B115B16069FFF708FF694220462C
:10327C0009B2BDE8F04105F044B86069414604F07C
:10328C00D8FF013EE5E7044A0821204605F04BF93A
:10329C00E0E700BF3CB200008AB4000013B58368BD
:1032AC008DF80710D3F860220446D00721D5D98FAA
:1032BC009A8F8A421DD0481C19449DF80720D88744
:1032CC0081F84220D3F86012890710D5D3F8603208
:1032DC0060690B4913F0040F18BF2A2204F0A9FFF0
:1032EC00204604F0C7FF10B16069FFF7C7FE02B0BB
:1032FC0010BD01220DF10701204605F021F9F6E77A
:10330C00AFB9000083680A4A1B6810B50446022155
:10331C0005F009F9A368D3F860329B0707D520465E
:10332C00FFF7DEFE2046BDE8104004F0C7BF10BD1D
:10333C008AB40000014905F062B900BFF2B2000086
:10334C002DE9F04F0E4600218BB0044617460D4672
:10335C0005AA304601F10108FFF75EFEB0B995B140
:10336C0027B13A460821204605F0DDF8224FDFF858
:10337C008CA0DFF88CB000214B1C05AA30460293C0
:10338C00FFF74AFE60B90BB0BDE8F08F006810B1D2
:10339C0005F0A5FC80B2854238BF05464146D7E70B
:1033AC000368D0F804900393384605F098FC039B0F
:1033BC0080467BB11A786AB1CDE9005352463B4640
:1033CC000821204605F0AFF8B9F1000F04D160696F
:1033DC00FFF7B0FF0299CFE75A4620463B4608213B
:1033EC0005F0A1F86A1C02EB480292B2494620464D
:1033FC0005F012F9EEE700BFDDB90000C4B900001A
:10340C00CBB90000F7B5064608680D46B8B105F013
:10341C0066FC84B20B4F384605F061FC2B680A4AF7
:10342C00009704440821304605F07DF8A4B2696881
:10343C002246304603B0BDE8F04005F0EDB8044636
:10344C00E8E700BFD9B90000BFB7000010B50749C5
:10345C00044605F054FC38B10549204605F04FFCF4
:10346C00B0FA80F0400910BD0120FCE7CFB9000094
:10347C00D2B9000010B58368D3F860329B060446BD
:10348C0003D50449406905F03EF9A368024A9A62E3
:10349C00002010BD629D00001800500008B5836923
:1034AC00034A1B68082104F081FC002008BD00BF02
:1034BC00E0B900007FB50F4E04460025A268E06815
:1034CC000DF10E0302F5A172012105F0A4F9BDF86E
:1034DC000E00A36850B103F5A173009332462B463E
:1034EC000821204604F062FC0135E7E783F842012D
:1034FC0004B070BDF0B90000022907B50DD15368B6
:10350C0001930E4B009313680D4A012104F04EFCFD
:10351C006FF0150003B05DF804FB8368094AD3F81B
:10352C00603213F0020F4FF00801074B18BF13461F
:10353C00064A04F03BFC0020ECE700BF07BA000091
:10354C00FEB9000054AC0000FAB900001CBA00002F
:10355C0010B58368D3F860329A06044603D5074940
:10356C00406905F0D0F8A368D3F860329B0603D508
:10357C000349606905F0C7F8002010BD699D000083
:10358C006E9D0000F0B5012985B004460DD053683E
:10359C000193594B00931368584A012104F006FC1F
:1035AC006FF01505284605B0F0BD8368D3F860327E
:1035BC009A0603D55249406905F0A5F86FF0F90158
:1035CC002046FFF761FDFA212046FFF773FDA06846
:1035DC0000254FF48072294600F5A1708DF80B5030
:1035EC0005F0DEFB4749606905F08DF8606904F071
:1035FC001AFC4FF47A766068036801221F690DF19A
:10360C000B0103ABB847039B53B9013E4FF47A70DF
:10361C00B6B206F019F9002EEDD16FF0850534E045
:10362C009DF80B30A1681B2B5AD091F842211B2A14
:10363C00E1D1522B54D10D44002385F8423191F83D
:10364C0043215B2A54D101F5A2751F46022615F8B9
:10365C00010B32463B2806F10106B6B22BD1B6F56A
:10366C00807FDAD002F2431211FA82F2002312F8B0
:10367C00015B55BBFA2B28BFFA23FA2F4B853B462F
:10368C0028BFFA2381F842510B85A368D3F8603226
:10369C009B0603D51C49606905F035F8002D81D0D7
:1036AC00A3681A4A9A620321194A204604F07EFB49
:1036BC006FF0070576E707EB870300EB4303303B1E
:1036CC00B6F5807F9FB2C2D1A7E703EB8303013627
:1036DC0005EB4305B6B2303DFF2EABB2C7D99CE724
:1036EC004A190135ADB2092D82F8423183D9002334
:1036FC0081F8423191E700BF07BA0000FEB9000023
:10370C00749D00002BBE0000789D00001800500036
:10371C002DBA00002DE9F04F074689B015468946B1
:10372C0021B90324204609B0BDE8F08F104605F0FE
:10373C0016F90028F5D04FF000084146022424E089
:10374C005C463CE029460AF5A17005F07EFA064677
:10375C0000284CD005F0C3FA82B2601C013231460D
:10376C00304405F0FAFA22465946304605F00DFB76
:10377C004FF020033355BAF8400001300444AAF846
:10378C00404008F10108002401994B1C03AA48464B
:10379C000193FFF741FC0646E8B131680022284648
:1037AC0004F05EF90028EFD1D6F800B0D7F808A0E5
:1037BC00BBF1000FC4D0584605F091FA84B2BAF8A8
:1037CC0040202244FF2ABDDD0A4A2B4603213846FD
:1037DC0004F0A9FE0124B8F1000FA3D0B8682A4662
:1037EC0000F1400100F5A17004F049FC9AE70224B5
:1037FC00F1E700BF30BE00002DE9F84305464FF05D
:10380C002003EFF3118683F31288BFF36F8F0E4BF7
:10381C001C689CB10D4FDFF838804FF00C09D4E9CF
:10382C000132002D08BF13462BB198F8142009FB68
:10383C0002F2B85C98472468002CF0D186F311880A
:10384C00BFF36F8FBDE8F883080900201009002032
:10385C008C0A00204209012300F01F0003FA00F03B
:10386C00074BBFF35B8FC04303EB820353E8002F7E
:10387C00024043E800210029F8D1BFF35B8F704769
:10388C001C09002038B51A4B1C7DBFF35B8F04F06C
:10389C001F0301229A40174B6109D04303EB8103AC
:1038AC0053E8001F01EA000543E8005CBCF1000F7F
:1038BC00F6D1BFF35B8F114213D00F4B0F4D8BB171
:1038CC000C236343EA18E85C517805F08EFA00206B
:1038DC00FFF792FF0C235C432A1900232B51C2E9FA
:1038EC00013338BD83F31188BFF36F8FEFE700BF4F
:1038FC008C0A002020090020F78D00001009002000
:10390C002DE9F843324B334A1C7DBFF35B8F6309BF
:10391C004FEA830952F823302F4EBFF35B8F04F02C
:10392C001F0843FA08F313F0010F07460AD10146AA
:10393C00204600F069F828B107C80C2303FB046388
:10394C0083E807000C236343F218F55C2DB920467D
:10395C00FFF780FF2846BDE8F8837B1C0FD0D2F818
:10396C0008C01E481E4A4FF4004500210023ECFB02
:10397C000501FCF7ADFB0121381A05F045FF02F0FB
:10398C00A1FE0120FFF738FFBFF35B8F012303FA81
:10399C0008F8144B994459E8003F43EA080349E8F6
:1039AC000032002AF7D1BFF35B8F0F4B33B10C23DE
:1039BC006343F218F05C517805F00BFAFFF762FFE5
:1039CC002046FFF747FF03F04DF80120C3E700BF87
:1039DC008C0A00201C090020100900203F420F0017
:1039EC0040420F0020090020DF8D0000054BBFF383
:1039FC005B8F53F82000BFF35B8F003818BF01209A
:103A0C00704700BF240900202DE9F04F85B00F4608
:103A1C0003A900F047F8DFF88080DFF880A0441E8F
:103A2C0024B24FF0000B631C04D10026304605B0C5
:103A3C00BDE8F08F039A04EB440302EB830612F803
:103A4C002300FFF7D3FF054610BB70684FF4004905
:103A5C00C4462946E0FB09C152465B466046FCF76A
:103A6C0037FB0190B068C4462946E0FB09C15B46B0
:103A7C0052466046FCF72CFB094B1B68591C01D0C5
:103A8C00834205D97A1CD1D0019B1844B842CDD9B8
:103A9C00013C24B2C7E700BF3F420F0040420F0079
:103AAC009400002008B9024B0B600020704700BF47
:103ABC0078A40000034B43F8302003EBC00359609B
:103ACC00704700BF3C010020014910220A6070477A
:103ADC0010ED00E072B6404080F31188BFF36F8F99
:103AEC00BFF34F8F30BF62B6BFF36F8F704700BF0D
:103AFC0072B6494081F3118820BF80F3118862B6F9
:103B0C00704700BF0028ACBF00F16040064B4FEA85
:103B1C004111ACBF00F5614000F00F00C9B2B4BF59
:103B2C00195480F80013704714ED00E043B2002BD9
:103B3C0008DB012200F01F0002FA00F05B09024AC8
:103B4C0042F82300704700BF00E100E0054B42093A
:103B5C0000F01F0053F82220012303FA00F010405C
:103B6C00704700BF00E100E030BFFFF7FDBF00BFB2
:103B7C000B4A08B50B4B22F07F029A60BFF34F8FB4
:103B8C00BFF36F8FD3F8882022F47002C3F888201B
:103B9C0002F0F2F903F09EF800F0D6F902F034FAD4
:103BAC000000000000ED00E00A4A0B499368096828
:103BBC00C3F8B0100949C3F8AC004B6843F080530C
:103BCC004B60002383F31188BFF36F8F9368D3F896
:103BDC00B00070478C0A0020E4A5000000ED00E066
:103BEC0013498A684FF030001044EFF3098C80E8D9
:103BFC00F01F202080F31288BFF36F8F0D4F4FF012
:103C0C000066CA698A603E60D2F8AC000023C2F834
:103C1C00AC3080F3118804B5104600F039FABDE8D9
:103C2C00044002F1300090E8F01F8CF309887047D3
:103C3C008C0A002004ED00E01EF0040F0CBFEFF323
:103C4C000880EFF30980816911F8021C0229FFD06A
:103C5C0001B504F0CAFE01BD42F8203C009B42F8BD
:103C6C001C3C0A49019B42F8183C029B42F8143C4C
:103C7C0021F001014FF0807342F8043C42F8081C1B
:103C8C000023203A0265C0F8AC3070472B75000059
:103C9C000A4A0346906878B113F1160FD0F89C00CD
:103CAC0005D0A0F120029A4205D8834203D281426A
:103CBC0028BF002070470020704700BF8C0A0020EE
:103CCC0008B5094B98600D46144600F0E1F9204602
:103CDC0085F30988002163B681F31188BFF36F8FD8
:103CEC000022002303F01BFC8C0A002001B572B6E5
:103CFC000B4A906900281EBF0021916105F06BFCF6
:103D0C0062B6EFF30580A0F110004FEAC000054940
:103D1C00014409C99847BDE8014003490847000020
:103D2C008C0A00203C010020393D0000044B9968AE
:103D3C00D869884203D003494FF080520A6070471B
:103D4C008C0A002004ED00E038B51C4B14469A6A2E
:103D5C009A6A9A6A0546900720D5586B9A6A120699
:103D6C001CD519B19A6A22F080029A629A6A9A6AF0
:103D7C009A6AD20615D49B6A9B0712D400200F4B6B
:103D8C009A6A920642BF5A6A22F400525A629A6A9E
:103D9C0042F0FF029A620023237038BD6FF01500C9
:103DAC00E4E7064B5B681905E8D52946FFF770FF79
:103DBC000028E3D080F309880220E0E700ED00E062
:103DCC000D4B9A6A9A6A9A6A920508D59A6B9A6A06
:103DDC00120404D518B19A6A22F400429A62064B76
:103DEC009A6A9A6AD20558BF9A6A9A6A002042F473
:103DFC007F429A620870704700ED00E070B5484B46
:103E0C005B688AB00D46C3F30803002686F311885D
:103E1C00BFF36F8F02F07F41B1F17F4F11D102F0F0
:103E2C000C0108290DD0110701D4054601260022EA
:103E3C00033B8DF80720032B6BD8DFE803F0045508
:103E4C00595D3546F3E7364BDC6A14F0020460D159
:103E5C00DA6A002A15DBDA6A520012D5AA6932F83E
:103E6C00021C4DF6027291420AD093F828200AB334
:103E7C000DF1070201212846FFF766FF044600E01A
:103E8C002C689DF807309BB92022294602A804F023
:103E9C007CFF099B002E3ED0C3F3080222B96FEAC7
:103EAC0053236FEA4323099302A9204604F09BFD98
:103EBC000AB070BD93F829202AB10DF10701012039
:103ECC00FFF77EFFDAE75A8D92B2002AD9D09A6AB0
:103EDC009A6A9A6A9A6A9A6A9A6A9A6A6FEA024221
:103EEC006FEA12429A62CCE70DF107020021C2E799
:103EFC000DF107010020E3E7094B9A6A9A6A9A6A66
:103F0C009A6A9A6A9A6A9A6A6FEA02426FEA12424B
:103F1C009A620024B5E723F4FF7323F00103C2E790
:103F2C0000ED00E0024A536943F0100353617047FF
:103F3C0000ED00E0EFF30880EFF3098101B5724664
:103F4C00FFF75CFF01BD00BF044800232021C2180D
:103F5C000133272B82F80013F9D1704700E100E000
:103F6C00002080F31488BFF36F8F05F007FE00204C
:103F7C0011490860BFF34F8F104880F3088800F098
:103F8C0033F8202080F311880D484FF0AA014FF42C
:103F9C00026204F005FF0A484FF40261401880F3F6
:103FAC000988EFF314800221084380F31488BFF3CF
:103FBC006F8FFFF7DDFD000094ED00E0601D002029
:103FCC00E01E00200749D1F890200023C2F30722FD
:103FDC001846934200D17047C1F89830C1F8A00040
:103FEC000133F6E700ED00E008B572B6002383F369
:103FFC001388FFF7E7FF144B4FF0FF32C3F8802014
:10400C00C3F88420C3F88820C3F88C20C3F8902010
:10401C00C3F89420C3F89820C3F89C20C3F88021DF
:10402C00C3F88421C3F88821C3F88C21C3F89021EC
:10403C00C3F89421C3F89821C3F89C2162B6BFF34E
:10404C004F8FBFF36F8F08BD00E100E0084B9B68FA
:10405C0083420BD1EFF3058343B1064B5A6842F010
:10406C0080525A605A6A22F400425A6202F0CABD67
:10407C008C0A002000ED00E0024B034A03480121AA
:10408C0000F070B8000001200000002078A40000AF
:10409C00D0F89C20054B203A1A60054A2021C3E930
:1040AC0001121846012100F067B800BF400900203A
:1040BC0000000B15F0B51F4F00268E4201DB104699
:1040CC00F0BD44689CB353B104F1FF3C14EA0C0FEF
:1040DC0018D11F2C16D905681CEA050F12D1202CFB
:1040EC000568D0F808C0D2B20FD9B4F1004F0ED881
:1040FC00013CB4FA84F4C4F11F046400072A4CEAAE
:10410C00040406D96FF01502D9E70824F6E73E241B
:10411C00F4E725F01F05154345F0100544F00104A4
:10412C00C7F89820C7F89C500132C7F8A040013658
:10413C000C30C2E700ED00E0044B0522C3F89420DC
:10414C00BFF34F8FBFF36F8F704700BF00ED00E0E0
:10415C00BFF35F8F024B0022C3F89420704700BF5F
:10416C0000ED00E010B5034C01232278FFF7A2FF0D
:10417C00207010BDF70C002008B5094A00231278F6
:10418C00FFF798FF10F1160F02D0064A072800DD42
:10419C0008BDC2F89800C2F8A0300130F6E700BFA5
:1041AC00F70C002000ED00E014490868082810B551
:1041BC0021D8FFF7CDFF124C49680022904201F143
:1041CC000C0105D10F4B1870FFF7B6FF002010BD86
:1041DC00C4F8982051F80C3C23F01F03134343F010
:1041EC001003C4F89C3051F8043C43F00103C4F8AC
:1041FC00A0300132E2E74FF0FF30E8E784A4000082
:10420C0000ED00E0F70C0020014B1860704700BF78
:10421C00980000200CB41FB509B90DF10300CDE9CD
:10422C00020107AB069A0648019302A9FDF7A2F812
:10423C00029B00221A7005B05DF804EB02B07047C7
:10424C00C58D00004FF02003EFF3118283F3128829
:10425C00BFF36F8F06490123C1F840354FF0804101
:10426C00C1F8783582F31188BFF36F8F0020704747
:10427C0000E001404FF08043C0B2C3F81C05BFF30F
:10428C004F8F0549054BCA6802F4E0621343CB60BB
:10429C00BFF34F8F00BFFDE700ED00E00400FA050F
:1042AC0020B1034B800143F001031847704700BF56
:1042BC00809D0000084B70B5C31A0D4607499B1032
:1042CC00044659430648402204F0B1FD2B460146F2
:1042DC002046BDE8704018475C090020B76DDBB67E
:1042EC00EC9B000073B50C4C0C4A4023041B009350
:1042FC000D460B460A49A41061430646094804F0D2
:10430C00C2FD011E05DA30462B4602B0BDE87040F6
:10431C00184702B070BD00BF5C090020038F00007D
:10432C00B76DDBB6EC9B000010B505F08BFA4FF4C3
:10433C007A72A0FB0203074C02FB0131C00B40EA6E
:10434C004140C90BC4E90001BDE81040012001F057
:10435C0021B900BF38030020002270B501210446AA
:10436C00104604F046FB0F4801F004F90E4B98423E
:10437C0015D105F080F826690C49304603F073F826
:10438C0000280BDB246909490125356404F11C0064
:10439C0003F069F8002801DBE564002070BD6FF0C4
:1043AC000400FBE7F14300000000AD0B10A500007A
:1043BC0001460C2309484B4370B5C418D4E90E567A
:1043CC0000224033A263184404F01EFD2DB1324686
:1043DC002B460348BDE87040184770BD5C090020AF
:1043EC00EC9B000010B1012804D07047034B1B6CF0
:1043FC005B0701D1FFF7DCBF704700BF5C090020F1
:10440C0008B54FF02003EFF3118183F31288BFF34B
:10441C006F8F114A136843F0020013F00103106010
:10442C000CD04FF08042D2F80C34D2F80C2413F09C
:10443C00010303D0094804F0E7FC012381F3118840
:10444C00BFF36F8F23B1BDE808400020FFF7B0BF6A
:10445C00BDE80840FFF768BFAC0900209C090020AC
:10446C007FB500220123CDE9022304ABCDE904334F
:10447C00094ACDF800D06B46CDF804D004F034FDD9
:10448C00002805DB4FF480420023684602F09AF8BE
:10449C0007B05DF804FB00BF1B8F000010B5074C84
:1044AC0023782BB94FF4A57005F0CEF901232370B6
:1044BC00BDE81040002001F06DB800BFF80C0020E2
:1044CC002DE9F74F4FF080480546D8F8186406F4EC
:1044DC0080364FF02003EFF3118783F31288BFF37C
:1044EC006F8F05F0AFF94FF47A73A0FB034003FB19
:1044FC000100D8F80C94D8F80C34254BD3F800B044
:10450C00244BE40BD3F800A044EA404487F3118811
:10451C00BFF36F8F204ADFF88480214F2846082193
:10452C0003F044FC19F0010FDFF878901E4AB9F83B
:10453C001A300093284614BF43463B46082103F02B
:10454C0035FCA4EB0B03009328465B46174A082165
:10455C00A4EB0A0403F02AFC53462846144A0094A0
:10456C00082103F023FC2846124A082103F01EFC04
:10457C00B9F83630009328460B4A002E14BF434638
:10458C003B46082103F012FC002003B0BDE8F08F7D
:10459C00380300204003002096BE0000F3B2000058
:1045AC0091BE00005C090020A1BE0000BBBE000053
:1045BC00DDBE0000FEBE000010B505F043F94FF45F
:1045CC007A72A0FB0203074C02FB0131C00B40EADC
:1045DC004140C90BC4E90001BDE81040012004F0C2
:1045EC0057BF00BF40030020084BBFF35B8F53E85D
:1045FC00002F22F0020143E800100028F7D1BFF38E
:10460C005B8FD30701D4FFF7D7BF7047AC090020ED
:10461C00024AC3B21C2003FB002070475C09002037
:10462C002DE9F0413949BFF35B8F0746012251E870
:10463C00003F41E800200028F9D1BFF35B8F33B96C
:10464C00334934484B60CB608A6002F01FFF7B1EFD
:10465C00012B2FD8012F07D14FF08043D3F81C34F6
:10466C0003F00303012B25D004F09AFF044618B97C
:10467C00294B1B78002B41D14FF02003EFF311860F
:10468C0083F31288BFF36F8F0124DFF890804FF013
:10469C008045D5F81834D5F81824D2030CD503F07E
:1046AC000303012B01D0012F06D10CB386F3118823
:1046BC00BFF36F8FBDE8F081ACB13046FFF718FA4D
:1046CC00D5F81835002BE4D1D5F80421002AE0D018
:1046DC00C5F80431D5F804310123C5F81835C8F8EC
:1046EC008031AB60D5E70021212002F06BFAE7E7BF
:1046FC004FF080430222C3F80423DBE74FF08043E2
:10470C000222C3F808230646BFE700BFB009002009
:10471C004C090020780900202911002000E100E05C
:10472C000A2838B5064D044603D128680D2104F03B
:10473C00F1FB2868E1B204F0EDFB204638BD00BF68
:10474C00B409002008B5084B0848186004F0E7FECF
:10475C0038B10748FFF758FD0548FCF717FD002056
:10476C0008BD6FF01200FBE7B40900201C9C000090
:10477C002D47000030B54068047B01F01F05B2F5F1
:10478C00001F45EA441585B04FF0000404D12846BB
:10479C0001F0BAF900202EE0B2F5800FCDE9024409
:1047AC002BD1B3F1007F0CBF042305238DF8083007
:1047BC00836823FA01F1C9072BD4B2F1A07F28D169
:1047CC0005F01F0303F5E0734FF0A04252F82330BD
:1047DC00DB071ED40DF107042146284601F0FCF836
:1047EC00144B984214D1204601F044F9124B9842D4
:1047FC000ED06FF00B0005B030BDB3F1C06F05D01B
:10480C00B3F1007F0CBF02230123CFE70323CDE7D5
:10481C0003940023194602AA284600F0B5FF064B64
:10482C00984204D10121284601F02AF9B2E76FF031
:10483C000400E0E70400AD0B0000AD0B10B501F077
:10484C0009F9044668B901F0DDF8084B98420AD121
:10485C000748214601F0BAF822460521062004F04B
:10486C00C8F8002010BD6FF00400FBE70000AD0B92
:10487C0081480000430970B510D1094B596869B1E2
:10488C0001250C68074E85408A682A4002D04B6887
:10489C003046984714B121462468F5E770BD00BF37
:1048AC00B8090020049C00002DE9F04347683B7BCD
:1048BC0001F01F0585B00E4645EA43151446CAB9EA
:1048CC0002A9284601F088F80446284601F044F96C
:1048DC004A4B984204D06FF0040005B0BDE8F08359
:1048EC00844205D19DF8080001F0BEF8A042F2D137
:1048FC000020F2E74FF000090DF103013046CDE93D
:10490C00029901F069F84B46804602AA49462846AE
:10491C0000F03AFF394B984202D06FF01500DCE7FB
:10492C00804503D19DF8030001F09EF8A30351D5F7
:10493C0040F20663234040F2062293423BD00CD84F
:10494C00062B15D004D89BB1022BE6D104230FE023
:10495C00B3F5007FE1D101230AE040F20242934219
:10496C002BD0B3F5C06F2AD0B3F5806FD5D102230D
:10497C008DF8043084F48033C3F30043E0068DF8E3
:10498C00053054BFC4F34013032321038DF80630C4
:10499C0017D57B68012101FA06F6C3F808650022D9
:1049AC0001A9284600F09AFF144B984214BF6FF0EF
:1049BC001500002091E70723DAE70523D8E7032346
:1049CC00D6E7620341BF7B68012101FA06F6C3F802
:1049DC000C65E4E7E3064FF0000354BFC4F3401446
:1049EC0003241A4601A928468DF8044000F0CCFE99
:1049FC00024B98423FF47CAF8FE700BF0000AD0B39
:104A0C0070B54B79012B20D18B79032B1DD1CC792F
:104A1C000CB1012C19D10A7912B1022A15D10E222E
:104A2C000B684568B3F5164F2D6862D02BD8B3F5DB
:104A3C00165F61D014D8B3F5966F5FD008D8B3F574
:104A4C00967F5ED0B3F5167F5ED06FF085004FE099
:104A5C00B3F5166F5BD0B3F5965FF6D1364B3CE0F1
:104A6C00B3F5E14F56D007D8B3F5615F54D0B3F529
:104A7C00964FEAD1314B30E047F61226B342E4D1DF
:104A8C004FF4000329E0B3F5613F47D013D8B3F5D9
:104A9C00963F46D009D84DF6C026B34243D0B3F565
:104AAC00614FD2D14FF46B0317E0B3F5E13FCCD19A
:104ABC004FF0EB7311E0B3F5612F37D008D8204ECF
:104ACC00B34236D0B3F5E12FBFD14FF0E86304E029
:104ADC001C4EB342B9D14FF080530069C5F8243550
:104AEC00031D03C92243C5F86C2583E8030000208D
:104AFC0070BD4FF41D03F0E7134BEEE74FF49E230C
:104B0C00EBE74FF4A033E8E74FF41C33E5E74FF441
:104B1C001D23E2E70D4BE0E70D4BDEE74FF06C7326
:104B2C00DBE70C4BD9E74FF46503D6E74FF0706326
:104B3C00D3E74FF08063D0E700B0130000A04E0025
:104B4C0090D0030040420F000050270000C07500B9
:104B5C0000F03A0000903A012DE9F7430746002295
:104B6C000121022003F045FF0220FEF7DFFFD7F8FA
:104B7C0004803E69D8F80040D8F80C900021C4F8A5
:104B8C00001501AA3760484604F092FB051E56DB5F
:104B9C00019BD9F800201979186804F0CBFB051E8D
:104BAC004DDB311D3846FFF72BFF0546002846D15B
:104BBC00D8F80430990719D506F1160001F096F8CB
:104BCC00224B98423FD1B07DC30003F1804303F5E3
:104BDC00F83304F10C0204F59071C3F81015C3F806
:104BEC0014251B4A01238340C2F804350823C4F85A
:104BFC00003598F808305BB9C4F81031D4F810318E
:104C0C0006F11503C4F834350123C4F83835236094
:104C1C00D8F804309A075CBF4FF48072C4F80423B0
:104C2C00DB0644BF4FF48003C4F80433143600236E
:104C3C00C4F84465C4F848350123A360E3602846F2
:104C4C0003B0BDE8F0836FF00405F8E70000AD0B8E
:104C5C0000F00140F8B5066905460F4604F0A0FCCB
:104C6C0010B9204B1B7883B94FF02003EFF311845C
:104C7C0083F31288BFF36F8F686804F067FA28BB60
:104C8C0084F31188BFF36F8FEEE76424686804F037
:104C9C005DFA70B9012004F0ECFB013CF6D1002167
:104CAC00212001F08FFFF0E784F31188BFF36F8FA1
:104CBC00F5E74FF02003EFF3118483F31288BFF371
:104CCC006F8F686804F042FA0028EDD0314601225B
:104CDC0001F8147F686804F01EFA84F31188BFF39E
:104CEC006F8FF8BD2911002010B501238340114AA4
:104CFC00BFF35B8FDC4352E8001F01EA040C42E86F
:104D0C0000CEBEF1000FF6D1BFF35B8F4FF48032B3
:104D1C0002FA00F002F1804202F58052C2F8080358
:104D2C00BFF35F8FBFF36F8F0B4214BF01200020C6
:104D3C0010BD00BFC80900201949F8B5044622F07F
:104D4C007F450868C1E90023A5F50013101AB3F5D7
:104D5C00400F22D2134B1B681A0A1B065E19124B0A
:104D6C0042F10007C3E90067012602F091F8A300A5
:104D7C0003F1804303F58833D3F84025AA420BD1C5
:104D8C001EB94FF40002C3F84025084B4FF4803095
:104D9C0000FA04F4C3F84443F8BD0026E5E700BF6D
:104DAC0060030020CC0900204803002000100140C3
:104DBC0019B3BFF35B8F0123104A834052E8001FE5
:104DCC00194342E8001CBCF1000FF7D1BFF35B8F15
:104DDC000B4A4FF480338340C2F80433094BBFF3C2
:104DEC005B8F1B68BFF35B8F23FA00F0C30742BFD6
:104DFC00054B4FF40032C3F800217047C80900205E
:104E0C0000100140C409002000E100E00D4B1868BF
:104E1C00010A0006BFF35F8F0B4BD3F8043518184B
:104E2C0041F10001B3F5801F0AD2084BD3E90023EE
:104E3C00904271EB030303D210F1807041F1000139
:104E4C00704700BFCC09002000100140480300202F
:104E5C002DE9F04F85B0164698460546FFF744FFFE
:104E6C000090FFF7D3FFB04271EB080378D2464BAA
:104E7C00301A68EB0101984271F1000380F08180D7
:104E8C00424B03EB0513D3E902ABD84508BF56459B
:104E9C0051D04FEA850909F1804905F1500709F510
:104EAC008839BF004FF4803101FA05F3BFB226F008
:104EBC007F4207F180470193D9F84005344B07F541
:104ECC0088371446D3F80415401A20F07F4021F09F
:104EDC007F4C0128C9F840C507D1CDE90221132028
:104EEC0004F0B2FCDDE90221294B01F1020CA4EB28
:104EFC000C0020F07F40B0F5000F88BF6446002006
:104F0C00386038680198C3F8440324F07F40C9F82E
:104F1C004005D3F80405814206D0201A023820F04F
:104F2C007F40B0F5000F19D8A41A24F07F4414EB7D
:104F3C00060A48F1000B15490E982B0101EB0512DE
:104F4C00C2E902ABC8500F9B53600024284600995D
:104F5C00FFF72EFF204605B0BDE8F08F2046B1E7E5
:104F6C0001230C4ABFF35B8FAB4052E8001F19437F
:104F7C0042E800100028F8D1BFF35B8FB246C3465D
:104F8C00D9E76FF01504E1E70100000150030020A0
:104F9C0000100140C409002073B5194B194D0024B1
:104FAC004FF0FF304FF0FF31C5F80845C3E902015F
:104FBC004FF48033C5F80433134B02264FF4003200
:104FCC000121C5F804631120C3F88021224603F0A7
:104FDC0010FD1120FEF7AAFD0C4A0123AB602B60DB
:104FEC0013600B4B0B4A0093019400232046FFF7F0
:104FFC002FFF3046FFF714FB204602B070BD00BFF8
:10500C00500300200010014000E100E0C80900201E
:10501C00454D0000FFFF7F002DE9F743354CD4F8D8
:10502C0004339A070BD5D4F8043143B1324A002328
:10503C00C4F80431D4F804311368013313604FF011
:10504C002003EFF3118283F31288BFF36F8FD4F830
:10505C000433DB0312D5BFF35B8F284B53E8001FDF
:10506C0021F0010043E80006002EF7D1BFF35B8F5F
:10507C00002936D1D4F84031002B32D1002382F3F1
:10508C001188BFF36F8F4BB3FFF7C0FE4FF02003B7
:10509C00EFF3118C83F31288BFF36F8F184BD3E9A6
:1050AC000267B04271EB07024FF0000220D34FF0C1
:1050BC00FF384FF0FF39D3E90015C3E902891A60B4
:1050CC004FF48033C4F848338CF31188BFF36F8FDF
:1050DC0021B1009532463B460020884703B0BDE81D
:1050EC00F0830023C4F84031D4F840310123C6E7E3
:1050FC001146E9E700100140CC090020C40900204A
:10510C0050030020431C13B521D0012821DDB0F53C
:10511C00000F20DA441EFFF779FE104BD3E9001381
:10512C00401AB0F5000F28BF0024013002190C48BA
:10513C00824228BF024652184FF0000009490190E4
:10514C00009143F10003FFF783FE02B010BD044849
:10515C00E0E70024DFE7024CDDE700BF600300203E
:10516C00FFFF7F00454D000008B5FFF74FFE024BD7
:10517C001B68C01A08BD00BF600300204FF07043CD
:10518C0093F8E02F062A09D1D3F8E83FC3F30313B1
:10519C00033B042B02D8024AD05C704700207047B6
:1051AC0063BF0000024AD2F80034002BFBD07047DA
:1051BC0000E0014010B504F04DF940B14FF08053C0
:1051CC00904AD3F82433C3F30423C2F84035FFF7D5
:1051DC00D5FF10B18C4B8D4A5A6704F03BF948B19E
:1051EC004FF080534FF08042D3F84432C3F3423334
:1051FC00C2F83C35FFF7C2FF30B1854AD2F8FC301B
:10520C0023F08073C2F8FC3004F024F940B14FF065
:10521C0080430022C3F80C21C3F81021C3F83825B1
:10522C00FFF7ACFF20B14FF080430322C3F8A02559
:10523C00FFF7A4FF60B1774B0522C3F810260122BB
:10524C00C3F888260022C3F818263F22C3F8142678
:10525C004FF08053D3F83021511C09BF4FF07043ED
:10526C00D3F8343193F8E02FD3F8E83F08BFC3F3F9
:10527C000313062A4DD1033B042B03D8664AD35C97
:10528C00002B46D04FF08052644BD2F80414C3F874
:10529C002015D2F80814C3F82415D2F80C14C3F84E
:1052AC002815D2F81014C3F82C15D2F81414C3F81E
:1052BC003015D2F81814C3F83415D2F81C14C3F8EE
:1052CC004015D2F82014C3F84415D2F82414C3F8AE
:1052DC004815D2F82814C3F84C15D2F82C14C3F87E
:1052EC005015D2F83014C3F85415D2F83414C3F84E
:1052FC006015D2F83814C3F86415D2F83C14C3F80E
:10530C006815D2F84014C3F86C15D2F84424C3F8CD
:10531C00702504F09FF848B14FF080534FF0804255
:10532C00D3F8583203F04F03C2F8E43E04F092F87D
:10533C0048B14FF08043D3F80024D20744BF6FF03C
:10534C000102C3F800244FF08053D3F83021062A11
:10535C0026D1D3F83431033B042B02D8304AD35C2A
:10536C0063B1304AD2F83C3743F48063C2F83C371F
:10537C004FF08053D3F83031062B11D14FF08053BE
:10538C00D3F83431033B042B02D8274AD35C3BB10E
:10539C004FF01023D3F808224FF08043C3F8582560
:1053AC004FF01023D3F80022002A03DBD3F8043289
:1053BC00002B22DA1D4901234FF01020C1F80435CF
:1053CC001524FFF7EFFEC0F80042FFF7EBFEC0F824
:1053DC000442FFF7E7FE0023C1F80435FFF7E2FEB5
:1053EC00BFF34F8F0A49124BCA6802F4E0621343B1
:1053FC00CB60BFF34F8F00BFFDE70E4B0E4A1A6018
:10540C0010BD00BF0030014000C007400DF0ADBA28
:10541C0000ED00E00050004054BF000000C0004010
:10542C0059BF0000001000405EBF000000E00140CA
:10543C000400FA05C80000200090D00370B50125C7
:10544C000268B2FA82F3C3F11F035E1CDCB214D003
:10545C00BFF35B8F05FA03F322EA030350E8006FF6
:10546C00964204D140E8003CBCF1000FF6D1BFF3EA
:10547C005B8FE5D102480C7070BD0248FCE700BFA1
:10548C000000AD0B0200AD0B0368CB40DB0710B581
:10549C0015D4012303FA01F10368BFF35B8F41EAD2
:1054AC00030250E8004F9C4204D140E8002CBCF1B0
:1054BC00000FF6D1BFF35B8FEED1024810BD02484E
:1054CC00FCE700BF0000AD0B0400AD0BF7B50446C4
:1054DC0018B1012829D003B0F0BD4FF0804302224F
:1054EC00C3F80823C3F80401D3F804210122DA60BD
:1054FC0001239C428DF8073014BF00250DF10705E0
:10550C0042F210774FF08046D4B1012CE3D125B193
:10551C00D6F80C3403F001032B70D6F80C34DB03F3
:10552C0018D4134B00225A71D5E74FF08043002258
:10553C00C3F80803C3F80021D3F800215860D7E75B
:10554C0025B1D6F8183403F003032B60D6F81834C1
:10555C00DA03C0D52DB9012003F08BFF013FD3D165
:10556C0003E09DF80730012BF5D0012CD9D0B2E720
:10557C00D0090020044B1A7922B9012218609A80B4
:10558C000248704702487047D00900200000AD0B5C
:10559C000C00AD0B38B510B1012844D038BD4FF01C
:1055AC008042D2F81814D2F8183413F480330BD18B
:1055BC00D2F81414C90710D5D2F81C349B0708D4A0
:1055CC000223C2F80433E9E701F00303012B04D0F2
:1055DC001BB10020FFF77AFF00234FF08042C2F886
:1055EC0018350023C2F80431D2F804310223C2F872
:1055FC000433124AD2F8FC0040F08073C2F8FC303D
:10560C000F4B1C6844F0010119605D685968491B17
:10561C00B1F50A5FFAD31C604FF08043C2F8FC006E
:10562C0001229A60BAE74FF080430022C3F80021B0
:10563C00D3F80021C3F804031860AFE700ED00E0D5
:10564C00001000E04FF0804310B5D3F800216AB190
:10565C000022C3F80021D3F800210122C3F808234B
:10566C00114B587910B95A711B6898474FF0804309
:10567C00D3F8042172B10022C3F80421D3F8042119
:10568C00D3F81824D3F81814920704D10122C3F8C4
:10569C0018259A6010BD0222C3F80823024BBDE8FE
:1056AC0010401B6801201847D0090020034B08301C
:1056BC0033F81000C0F34010704700BFCC0000203E
:1056CC0070B500F108030C4C34F81330DA050546BC
:1056DC000E4607D5C3F3432304EBC30254F833300F
:1056EC0052689847A3682BB1E26831462846BDE85A
:1056FC007040184770BD00BFCC000020124A083023
:10570C0010B432F81030D9051BD5C3F3432123F460
:10571C00F85322F8103002F11004002034F8023B48
:10572C0013F4807F03D0C3F34323994209D0013093
:10573C002028F3D1002342F83130044810BCFFF785
:10574C00A3BE10BC704700BFCC000020200100207D
:10575C0038B50246FFF7AAFF094C02F1080540B123
:10576C0034F8153007495B0B03F5A273002041F8A0
:10577C0023001046FFF7C2FF002324F8153038BD74
:10578C00CC000020006000402DE9F34104461E4689
:10579C0009B34D4F00F1080837F81850AB0706D580
:1057AC00FFF784FF18B1494802B0BDE8F08104F05E
:1057BC001F00800000F1A0400978D0F8003725F0D8
:1057CC00020523F00F0345F0010543EA810327F896
:1057DC001850C0F8003792B13B4B1578526804F161
:1057EC00080033F810108F070CD5002ADBD133F8E2
:1057FC00102022F01C0242EA850223F81020CEBBB6
:10580C003348D1E721F02001C904C90C23F810104A
:10581C00002AECD0032DC6D817782DB92D4A07F5E0
:10582C00A27142F82150E2E7BA0002F1804202F57F
:10583C00C04241EA4731D2F810C52CF0030CC2F833
:10584C0010C5D2F810C52CF4473C2CF4407CC2F89F
:10585C0010C5D2F810E54FEA042C0CF4F85C4EEAB3
:10586C00054E4CEA0E0C41F0200123F81010C2F842
:10587C0010C5BCE7D6E900762046FFF73FFF002FA6
:10588C00BED0114D2B689F4204D16B689E4201D152
:10589C00002209E010480DF10701FFF7CFFD0C4B7A
:1058AC00984281D19DF8072045F8327005EBC20370
:1058BC0008345E6035F8143043EA422343F48073B5
:1058CC0025F814309CE700BFCC0000200400AD0B81
:1058DC000000AD0B0060004020010020F8B504462C
:1058EC0071B3374E00F1080736F81750AB0704D4E4
:1058FC00FFF7DCFE08B13348F8BD15F01C0F4B78F0
:10590C0001D0012BF7D004F01F00800000F1A04063
:10591C0091F800E0D0F800C789785B002CF4E16CBA
:10592C0043EA0E232CF0070C43EA0C0343EA8103F1
:10593C0045F0030543F0010326F81750C0F8003773
:10594C000AB92148D8E71E4E04F1080736F81700AB
:10595C008307D0D592F800C06146890020F0200062
:10596C0001F18041C00401F5C041C00C26F81700BC
:10597C000023C1F810355578002DE2D0D1F8103540
:10598C00927823F4981323F4F853C1F81035D1F816
:10599C0010E5230203F4F8532D0443EA0E0305F437
:1059AC00403512052B4302F4801240EA4C3013436D
:1059BC0040F0200026F81700C1F81035C1E700BFF1
:1059CC00CC0000200400AD0B0000AD0B014BC3E973
:1059DC0002017047CC00002008B50246FFF766FEB6
:1059EC0038B1054B0548083233F812305B0B0B709D
:1059FC0008BD0348FCE700BFCC0000200000AD0B45
:105A0C000400AD0B38B50F4C94F85850BDB940227A
:105A1C00294604F1100003F0C3F90620FEF786F8BE
:105A2C00094B0A48C3F87C51D3F87C214FF0004253
:105A3C00C3F80423012384F85830636538BD044847
:105A4C00FCE700BFCC000020006000400000AD0B64
:105A5C000500AD0B034B93F85800003818BF01201C
:105A6C00704700BFCC00002001460148FFF70CBD79
:105A7C001C01002001460148FFF7E0BC1C0100207E
:105A8C0010B50246FFF712FE02F108041C4B33F866
:105A9C001430E0B113F0020419D15B0B9A0002F13F
:105AAC00804000F5C24002F1804202F5C042046021
:105ABC000068D2F8100540F00100C2F8100529B1B9
:105ACC00012202FA03F30F4AC2F8043310BDC3F3E8
:105ADC008203042B10D0052B10D04FF0A043D3F829
:105AEC00101502F01F03D94001F001010231BDE88D
:105AFC001040104603F0CEBC0321F8E70221F6E774
:105B0C00CC0000200060004008B50246FFF7CEFD37
:105B1C00C0B102F108010E4B33F81130990711D4C2
:105B2C005B0B01229A409B000A4903F1804303F569
:105B3C00C043C1F80823D3F8102522F00302C3F8A0
:105B4C00102508BDBDE808400021104603F0A2BC9A
:105B5C00CC000020006000400D4B00F1080210B595
:105B6C0033F81230DB0704460FD5FFF7CDFF204684
:105B7C0004F01F04FFF7ECFD04F5E0744FF0A043B4
:105B8C00022243F82420034810BD0348FCE700BF61
:105B9C00CC0000200000AD0B0400AD0B2DE9F74F3D
:105BAC004E4B4F484F49002501222C461E6836B1FA
:105BBC00D0F8046316421EBF1C601E6815430433E4
:105BCC008B424FEA4202F1D1454BD3F87C31BBB149
:105BDC004FF0A046D6F820350193C6F8203501AF1A
:105BEC004FF00108019C6CB93D4BC3F87C41D3F8D4
:105BFC007C31D6F820350193C6F82035002BEED138
:105C0C00012466E094FAA4F4B4FA84F4364A04F15C
:105C1C000803E00832F8131004F0070308FA03F243
:105C2C003B5C23EA02033B54A30003F1A049C1F3FC
:105C3C00820AD9F80027CB06D346C2F3014218D505
:105C4C00594620465FFA82FAFFF73AFDD9F8003739
:105C5C00C3F301439A4507D10021204603F01AFCF7
:105C6C005146204603F016FC08FA04F4C6F8204509
:105C7C00B8E7022A0CBF03210221204603F00AFCDC
:105C8C00BAF1030F04D0022A07D1BAF1010FEBD1FC
:105C9C0059462046FFF714FDE6E7032AE4D1BAF192
:105CAC00020FF4E795FAA5F3B3FA83F304FA03F2BF
:105CBC009B0003F1804303F5C04325EA0205D3F8AA
:105CCC001005D3F81015C0F30420C1F30141FFF700
:105CDC00F7FC002DE6D103B0BDE8F08F0061004069
:105CEC000060004020610040CC00002001460148CB
:105CFC00FFF7A4BB28010020F8B50779224E0C460B
:105D0C000C21794305467018037A002B3AD1725056
:105D1C0062684260697928689C46DAB2914229D857
:105D2C0040F30730FDF702FF2B686278D3F80415B7
:105D3C00164821F0030102F003020A43C3F80425BC
:105D4C00D3F80815A27821F0030102F003020A43EC
:105D5C00C3F80825D3F81015227821F00F0102F0B2
:105D6C000F020A43C3F810250C2303FB076601231B
:105D7C003372F8BD9A0002F5A072013340F802C0EC
:105D8C008258CAE70248F4E7D80900200000AD0B9E
:105D9C000500AD0B036801221A600279034B0C213C
:105DAC0001FB023302221A72704700BFD80900208F
:105DBC00036801221A610179024B0C2000FB0133AC
:105DCC001A727047D80900202DE9F0410E4C0F4F84
:105DDC000F4E00254FF48038236873B1D7F8043385
:105DEC0008FA05F21A4208D000232360A4F50040FB
:105DFC00236880B2D6E9003198470135042D04F1AF
:105E0C000404E9D1BDE8F0814081004000800040ED
:105E1C00D809002010B5144C144A154903232361EA
:105E2C006361144BA261E3614FF48063236200232E
:105E3C00A3626362E36222660F4A6266E01D10226F
:105E4C00A2662367E366636702F01FFFBFF35F8FF1
:105E5C000A49204602F019FFBFF35F8F2023A3717C
:105E6C00BFF35F8F10BD00BFE409002068BF0000C6
:105E7C0071BF0000290D0020190D002075BF000016
:105E8C002DE9F84FDFF848A0124D9B46A5EB0A050B
:105E9C00114BED1080460F4691465D430026BE42E5
:105EAC0002D13046BDE8F88F38F91640002C0DDDD4
:105EBC00A5420BD3013C24B204EB44040AEBC4000E
:105ECC005946C8470028EDDB0136E8E70020F7E724
:105EDC00EC9B0000349C0000ABAAAAAA0E4B70B538
:105EEC0053F82040013053F82060A64200D870BD12
:105EFC00D4E900352846984765B1EB6830B10028E5
:105F0C00B8BF4042FF28A8BFFF2018705A7842F053
:105F1C0001025A700834E8E7D0A50000034A044B8C
:105F2C0002609B1A0348DB1058437047EC9B00003F
:105F3C00349C0000ABAAAAAA014B98689830704711
:105F4C008C0A002008B50A4B012202201A70FFF7B8
:105F5C00C5FF01F095F80320FFF7C0FF00F0D4F95E
:105F6C00FAF724FA034A137B23F00103137308BDD9
:105F7C00291100202004002008B50348034A002101
:105F8C00121A03F009FB08BD800200202C1100201E
:105F9C0070B5174E174D184986B0B82303FB006631
:105FAC00164B059301220F23CDE903320023CDE9D3
:105FBC000133182303FB005504464FF4B07000FB6B
:105FCC0004110F4B00954FF4A072304600F008F905
:105FDC00737B0C482C7523F0040373734FF402632A
:105FEC0003FB04041C44EE606C6006B070BD00BF83
:105FFC00680300208C0A0020801D00207CBF00005C
:10600C00D5630000E01E002080B52D4BB4B083F3A7
:10601C0008882C4D2C4E6B692C4F43F400730024D4
:10602C006B61E02385F82230EC772C766C76AC76BD
:10603C0085F820406B6A43F4E0236B6285F82340BB
:10604C00FDF770FFFDF740FD4FF0FF33AB62EB62E5
:10605C00FEF7AAF8FEF710F840F20113ADF8243061
:10606C0006ABB360CDE92D44309403F057FA2046CB
:10607C00FFF734FF0120164DFFF730FF00F00EFD47
:10608C00144BF5610593012313490094CDE90343A7
:10609C004FF480623B46CDE90144284600F0A0F85D
:1060AC006A7B064622F0040228466A7303F0F4FA6F
:1060BC002046FFF76DFF3A4631462846FDF700FEB5
:1060CC000027002000ED00E08C0A0020515F00004A
:1060DC002004002081BF000060190020F8B505469F
:1060EC000E464FF02003EFF3118783F31288BFF3B2
:1060FC006F8F064B9C6A24B987F31188BFF36F8F9F
:10610C00F8BD20463146A847646FF4E78C0A00209E
:10611C004FF02003EFF3118183F31288BFF36F8FDD
:10612C00094A936A834207D15B6F936281F31188AA
:10613C00BFF36F8F70471346002BF7D05A6F824214
:10614C00F9D1426F5A67F1E78C0A002010B504466A
:10615C0008B9054B9C681F2204F1780002F09FFDE2
:10616C00002084F8970010BD8C0A0020437B102B74
:10617C000ED8102B1CD8DFE803F01D09131B151BC0
:10618C001B1B171B1B1B1B1B1B1B19000B487047D6
:10619C00202B11D00A4A0B48802B08BF10467047A1
:1061AC0009487047094870470948704709487047C3
:1061BC00044870470848704708487047AEBF000055
:1061CC00BDBF000086BF00008EBF000096BF000060
:1061DC009FBF0000A4BF0000F3B20000B4BF0000DA
:1061EC002DE9F04F85B0984600F15803C0E91633FD
:1061FC000732129B037322F0070A0423002501F1D6
:10620C00200B43730AF12007119B85600446C0E9FB
:10621C0006550E468373C5730F445246AA21584641
:10622C00DDF84C9002F0BCFD109B02930F9B019388
:10623C000E9B0093C4E927BA4346C4F8A4503A46CF
:10624C0031462046FDF708FD0E9BA3660F9BE366C7
:10625C00109B6565C4F8648023674FF02002EFF350
:10626C00118382F31288BFF36F8F104EB26A62678C
:10627C00B46283F31188BFF36F8FB9F1000F11D0A3
:10628C001F22494604F1780002F009FD84F897506A
:10629C00B3680BB1D3F8A830C4F8A830384605B0B1
:1062AC00BDE8F08F84F87890F2E700BF8C0A0020EC
:1062BC00F0B587B000270597109F04970F9F0397A1
:1062CC000E9F0297DDE912650D9F01970C9F0097B9
:1062DC000446FFF785FFB5F1FF3F08BFB6F1FF3F5E
:1062EC0005D055EA060305D1204600F0D1FA204628
:1062FC0007B0F0BD034932462B4604F1180000F0FC
:10630C004DFDF4E7C59600002DE9F043294C2A4DCC
:10631C0087B02646AE4204F130040FD300F0D2F918
:10632C00244CDFF898904FF4004640F2E737AC422B
:10633C0020D307B0BDE8F04300F094BB54F8043C04
:10634C00059354F8103C049354F8143C039354F8FC
:10635C00183C029354F81C3C019354F8203C0093D5
:10636C0054E90C0154E90A23FFF73AFF54F8303C86
:10637C005E65CEE7636A5A1C0DD023EAE3730021F5
:10638C003846C3FB060151EAC333D4F8008004D16C
:10639C00404600F07DFA3034C9E74FF47A7200239E
:1063AC00F9F796FE02460B4608F11800494600F034
:1063BC00F5FCF0E78002002080020020C59600006A
:1063CC00004870470063000308B50B4C0B4D4FF0B1
:1063DC002002EFF3118382F31288BFF36F8F03F067
:1063EC0003FA2B78A06113B9FDF774FBEFE7FDF707
:1063FC0087FA0028EBD1F7E78C0A0020291100203E
:10640C002DE9F341044617461E464FF02003EFF3E7
:10641C00118883F31288BFF36F8FC368324A6BB154
:10642C0080689168884219D057EA060318D188F31E
:10643C001188BFF36F8F6FF00F000CE0916891F92A
:10644C000E1021610133E3609368A36088F3118817
:10645C00BFF36F8F002002B0BDE8F0812169F0E737
:10646C0091F90E1090F90E309942A8BF19466FF0B1
:10647C007E029142B8BF11468B422EDD03F0B2F87A
:10648C000546CDE9007619482246414600F05CFAF3
:10649C000028E0D04FF02003EFF3118683F312882D
:1064AC00BFF36F8F236821699C420AD04BB193F9DB
:1064BC000E309942A8BF19466FF07E039942B8BFBF
:1064CC001946A06803F08EF800B945B1074831466B
:1064DC0000F0E6F86FF00A00BDE70025D1E786F37F
:1064EC001188BFF36F8FF5E78C0A00202A1100206A
:1064FC0038B583680446002B33D01D4A926893420A
:10650C0032D1DA7B013ADA73C368012B05D9013B2E
:10651C00C36000F0A7FA002038BD4FF02003EFF362
:10652C00118583F31288BFF36F8F0169806803F0C4
:10653C0059F8204603F00CF9A06060B190F90E20D8
:10654C0022610022C0F8B02003F0A6F809482946C1
:10655C0000F0A6F8DDE7E06085F31188BFF36F8FDC
:10656C00D7E76FF01500D7E74FF0FF30D4E700BF47
:10657C008C0A00202A11002038B504464FF0200365
:10658C00EFF3118583F31288BFF36F8F03F0E0F8FC
:10659C0050B10022C0F8B02003F07EF8294608481C
:1065AC00BDE8384000F07CB8D4E902329A4218BFFA
:1065BC000133A360022104F1100003F087FAEDE728
:1065CC002A11002013B54FF02004EFF3118184F34E
:1065DC001288BFF36F8F846844B1013C846081F3EF
:1065EC001188BFF36F8F002002B010BD52EA030474
:1065FC0006D181F31188BFF36F8F6FF00F00F3E7B3
:10660C00CDE900230246024800F09EF9ECE700BFFA
:10661C002A11002038B5074D2C6854B1FEF7A4FDA3
:10662C00054B04441C6128680021BDE8384003F088
:10663C00EBB838BDC00A00208C0A0020F8B504461F
:10664C000D464FF02003EFF3118783F31288BFF34D
:10665C006F8F104E00214FF4004C40F2E730316147
:10666C0000234FF47A72E4FB0C01F9F731FD002C96
:10667C00094B0ADC1860094BB0681D60FFF7CAFFB4
:10668C0087F31188BFF36F8FF8BD0228B8BF0220C3
:10669C00F0E700BF8C0A0020C00A0020BC0A0020D2
:1066AC0049B9EFF3058030B9054BDA699B689A421A
:1066BC0001D0FDF779BA81F31188BFF36F8F704762
:1066CC008C0A00204FF02003EFF3118183F3128822
:1066DC00BFF36F8F044B9A68D37B013BD37381F369
:1066EC001188BFF36F8F70478C0A002038B50246B3
:1066FC000C480D4D02F0CAFF044600B9EC68AB68BB
:10670C004AB95A7BD20606D1A26922B9DA897F2A04
:10671C0001D9EB6138BD9C4202D02046FFF77AFFCD
:10672C00EC61F7E7AC0A00208C0A002070B590F9F8
:10673C000D20437B002A014604DA03F07F034373E8
:10674C0002F05FFF4B7B154A63F07F034B73D2E97A
:10675C00083402F12005AB421BD0D3B191F90E6085
:10676C0093F90E0086420FD0801B00280CDD586870
:10677C00C1E90030016059609068431A5842BDE885
:10678C0070405841FFF7B2BFA34202D01B68002BE8
:10679C00E6D1C1E9005421605162EDE78C0A00207A
:1067AC0038B54FF02003EFF3118583F31288BFF354
:1067BC006F8F174B174A9C6811688C4207D1204683
:1067CC00FFF728FF85F31188BFF36F8F38BD0021C9
:1067DC001160114A1268C2B1E2897F2A15D8627B16
:1067EC00D20612D10D4A94F90E10126891420CDBAC
:1067FC000B4A944209D01A69824203DC2046FFF707
:10680C0095FFDCE7121A1A61DCE70022FBE700BFF8
:10681C008C0A0020B80A0020C00A0020BC0A002004
:10682C006803002070B490F90D20437B002A2ADB0A
:10683C00DA0628D1826932BB144A63F07F034373B2
:10684C00D2E9083402F12005AB4217D0B3B190F96C
:10685C000E6093F90E108E420BD0891B002908DDB7
:10686C005A68C0E900321060586070BC0020FFF715
:10687C003DBFA34202D01B68002BEAD1C0E90054F3
:10688C0020605062F1E770BC704700BF8C0A00209A
:10689C0010B54FF02002EFF3118482F31288BFF38E
:1068AC006F8F427B510704D484F31188BFF36F8F31
:1068BC0010BD22F004024273FFF7B4FF21460248D8
:1068CC00BDE81040FFF7ECBE2A11002008B590F986
:1068DC000D20437B002A014604DA03F07F03437347
:1068EC0002F08FFE044B9868431A58425841BDE899
:1068FC000840FFF7FBBE00BF8C0A00202DE9F041D9
:10690C00064615461C464FF02003EFF3118783F320
:10691C001288BFF36F8F02F0F1FE87F31188BFF37B
:10692C006F8FB4F1FF3F08BFB5F1FF3F08D02A4687
:10693C00234606F118000349BDE8F04100F02EBAD9
:10694C00BDE8F081C596000010B5074B9868074B61
:10695C000C4618601146DDE90223FFF7CFFF2046F5
:10696C00BDE81040FDF720B98C0A0020B80A0020C1
:10697C00F8B504464FF02003EFF3118683F3128829
:10698C00BFF36F8F437BDA0649B233D182698ABB7E
:10699C0003F07F03437302F034FE437B174A817389
:1069AC0063F07F034373104650F8203F83421BD0A3
:1069BC00D3B1576A93F90E50A94210D06D1A002D1D
:1069CC000DDD5A68C4E9003214605C600120FFF7E9
:1069DC008DFE012086F31188BFF36F8FF8BDBB428B
:1069EC0002D01B68002BE5D1536AC4E900031C607C
:1069FC005462EBE7A1730020ECE700BF8C0A002087
:106A0C0070B50446183002F0D9FE4FF02003EFF3B6
:106A1C00118683F31288BFF36F8F94F90D20637B7B
:106A2C00002A05DA03F07F036373204602F0E9FDC8
:106A3C000B4D637BA86843F010036373031B584230
:106A4C005841FFF753FE86F31188BFF36F8FAB6885
:106A5C00A34203D1BDE8704002F00EBE70BD00BF72
:106A6C008C0A002010B54FF02003EFF3118483F350
:106A7C001288BFF36F8F084B9A68D37B0133D373A3
:106A8C000020FFF733FE84F31188BFF36F8FBDE84E
:106A9C00104002F0F1BD00BF8C0A0020044B002115
:106AAC0003F12002C3E908220846FFF7C7BD00BF67
:106ABC008C0A0020F8B54FF02003EFF3118583F317
:106ACC001288BFF36F8F1A498868437B03F07F03EA
:106ADC00437302F096FD8B685A7B084662F07F0286
:106AEC005A7350F8202F82421CD0DAB14F6A93F9B6
:106AFC000E6092F90E40A6420FD0A41B002C0CDDA8
:106B0C005168C3E900210B6053600120FFF7EEFDD3
:106B1C002846BDE8F840FDF747B8BA4202D01268E3
:106B2C00002AE6D14A6AC3E9000213604B62ECE723
:106B3C008C0A002050EA01032DE9F04105460E466F
:106B4C0003D1FFF7B7FF002033E06FF00104241AE4
:106B5C004FF0FF3363EB0103012C73F1000302DAF6
:106B6C0002F06CFE44194FF02003EFF3118883F30D
:106B7C001288BFF36F8F104F104BB8681860FFF777
:106B8C00A5FEB8680E492A463346183000F006F9BF
:106B9C00BA68537B43F0100353734046FDF704F877
:106BAC0002F04CFE201A63EB0303012873F100037F
:106BBC00C9DBBDE8F08100BF8C0A0020B80A0020B8
:106BCC00C5960000B1F1FF3F08BFB0F1FF3F08B51B
:106BDC0006D1084B9868FFF713FF4FF0FF3008BD44
:106BEC00FFF7A8FF4FF47A7380FB0303C00B40EA56
:106BFC004340F4E78C0A0020014B9868704700BFB3
:106C0C008C0A00202DE9F04104464FF02003EFF3ED
:106C1C00118683F31288BFF36F8F437B1A0705D558
:106C2C0086F31188BFF36F8FBDE8F08123F020024B
:106C3C0042F00801D20923D14173A36813B1204655
:106C4C0002F0E7FC04F1180002F0B8FD04F158075B
:106C5C004FF00008A56DBD4200D0CDB90120FFF763
:106C6C0045FD2046FFF754FA104B9B68A342D7D141
:106C7C00EFF30583002BD3D13046FCF795FFCFE71C
:106C8C0003F05F0343F00803437302F0BAFCD4E74C
:106C9C00284602F0BEFC05F1180002F08FFDC5F885
:106CAC00B0802846FFF7BEFDD4E700BF8C0A002059
:106CBC00D3B5DDE90667089CCDE90067FFF744FE14
:106CCC001CB1034B9B685B69236002B0D0BD00BF55
:106CDC008C0A002008B50648064A0749121A02F029
:106CEC005DFCBDE80840054A0549064802F056BC63
:106CFC00000000208002002004C000000000000002
:106D0C0004C0000000000020034B1B680BB9FEF709
:106D1C002BBA0020704700BFC40A0020104B10B5DE
:106D2C001C689C4208BF0024FFF7EEFFA4B1D4E915
:106D3C0004321B1A62EBE070B3F1004F70F10002E9
:106D4C000ADA0028ACBF18460020064B1B6913B1A9
:106D5C009842A8BF184610BD6FF00040F5E700BF81
:106D6C002C0100208C0A002030B5036868B10A4A57
:106D7C005268904209D043B1D3E90421D0E90445CB
:106D8C00121941EB0501C3E90421426813605A60F2
:106D9C000023C0E9003330BD2C010020B3F1FF3FCC
:106DAC0008BFB2F1FF3FF8B504461F46154667D041
:106DBC0081604FF02003EFF3118683F31288BFF349
:106DCC006F8F6FF00102531B4FF0FF3C6CEB07030E
:106DDC00002B1BDB2B4BD3E90013521A6CEB030378
:106DEC00551B63EB0703012D73F10002BCBF01259A
:106DFC000023C0E904532448D0E9003C834218D155
:106E0C00C4E9000CCCF80040446026E0FFF77CFF9E
:106E1C00013547F100072D1847EBE077C4E904571B
:106E2C00E9E7521A65EB07059C45C4E90425E7D050
:106E3C001B68002BE4D0D3E90417D4E904258A425B
:106E4C0075EB070EEDDA8A1A67EB0505C3E9042525
:106E5C005A68C4E9003214605C60036883420BD04A
:106E6C009C4209D1FFF75AFF18B1084B1B698342AA
:106E7C0002D00021FEF746F986F31188BFF36F8F1D
:106E8C00F8BD00BFD80400202C0100208C0A002083
:106E9C002DE9F8430546FFF783FC4FF02003EFF391
:106EAC00118483F31288BFF36F8F244EDFF8908028
:106EBC003560244DD8F8000032684045D5E9001EF5
:106ECC004FEAE2770BD050B1D0E9043C9A4277EB11
:106EDC000C0916DA9B1A6CEB070CC0E9043C52182F
:106EEC004EEB0707C5E9002700253560FFF716FFB5
:106EFC002946FEF707F984F31188BFF36F8FBDE8BD
:106F0C00F88359184EEBE377D31A33600022002331
:106F1C00C0E90423C5E90017FFF726FF84F31188A5
:106F2C00BFF36F8F836898474FF02003EFF3118402
:106F3C0083F31288BFF36F8FBCE700BFC40A002035
:106F4C002C010020D804002010B54FF02003EFF3E3
:106F5C00118483F31288BFF36F8FFEF705F9054A8E
:106F6C00D2E90031C01841F1000184F31188BFF35C
:106F7C006F8F10BDD80400202DE9F3471D46294B17
:106F8C009F68012387F8603087F8613052EA050367
:106F9C0016460CBF0123002307F16002804602F065
:106FAC0086FC81464FF02003EFF3118A83F312889D
:106FBC00BFF36F8F97F8604064B901465246404664
:106FCC0002F046FD8AF31188BFF36F8F204602B0A2
:106FDC00BDE8F087002387F8603056EA050306D138
:106FEC008AF31188BFF36F8F6FF00A04EEE7CDE9D7
:106FFC0000650D4A0D485146FFF7A6FC04464FF0BC
:10700C002003EFF3118583F31288BFF36F8F2A46A9
:10701C004946404602F01CFD85F31188BFF36F8F83
:10702C00D4E700BF8C0A0020340100202A11002074
:10703C0038B503464FF02002EFF3118582F3128826
:10704C00BFF36F8FC160012181600068834206D15C
:10705C0085F31188BFF36F8F0024204638BDD0E92B
:10706C00003213605A600023C0E9003302F096FC32
:10707C00294604460148FFF713FBEEE72A110020CE
:10708C00024A0349034800F092B900BFF3B2000072
:10709C00C4BF0000D1BF000038B5064C064DAC4251
:1070AC0001D3002038BDD4E90112204602F029FD9D
:1070BC001434F4E780020020800200201FB5094B35
:1070CC00029302AB00240093074908488DF80C404A
:1070DC004FF0FF334FF4806200F0F0F8204604B01C
:1070EC0010BD00BFF8BF000000270020E004002006
:1070FC002DE9F04F474E85B004464FF0FF384FF066
:10710C00FF394FF02003EFF3118783F31288BFF39D
:10711C006F8FD4F8B8508DB9022104F1D00002F071
:10712C00F8FC002835D10023CDE90089029304F145
:10713C00C00239463848FFF7BBFDE2E7D4F8BC2063
:10714C002B68C4F8B830954201D1C4F8BC30D4F8DF
:10715C00D03043F00203C4F8D030EB6823F00403C2
:10716C0043F00103EB606B6887F31188BFF36F8FFB
:10717C00284698474FF02003EFF3118B83F31288C6
:10718C00BFF36F8FEB68990723F001020BD4EA6011
:10719C000EE004F1C80500220121284602F0F0FAA5
:1071AC000028F8D1BFE7306823F00303EB6070B917
:1071BC00D4F8D03023F00203C4F8D0308BF311880C
:1071CC00BFF36F8FD8059CD4FFF774FC99E70027A9
:1071DC00D0F800A03B464268954201460CD10168AC
:1071EC0097B972683160824200D1716040F8083BF7
:1071FC00FFF7C2F939460023BAF1000FD8D0504638
:10720C000F46DAF800A0E6E772683960904208BFD2
:10721C007760EBE7C80A00202A110020F8B5C36894
:10722C009A0704460E46C3F340051FD45F071FD4CC
:10723C000A680AB982680A60D80744BFA368336039
:10724C0037684CBF022501257FB31B4B9B68BB42A3
:10725C0011D102F0A5F980F00100C0B2D7F8D030FE
:10726C00D907C3F3800223D53AB140B96FF00F05AB
:10727C000023336013E00020F0E71B07F6D4002353
:10728C002360D7F8BC3063B9C7E92E44384602F006
:10729C004BFCE36843F00403E3603368A3602846C7
:1072AC00F8BD1C60C7F8BC40F0E76FF01505DFE7D0
:1072BC006FF01205DCE700BF8C0A0020F0B589B036
:1072CC0004460020C4E92E000E9D04F1C000C4E960
:1072DC00300004F1C800C4E932001DB3287900283D
:1072EC0040F2011008BF0120C4F8D00000204FF07C
:1072FC00FF364FF0FF37CDE90330CDE90100CDE982
:10730C000667094B00942046FEF7D2FF25B1296889
:10731C0011B12046FEF71AFF204609B0BDE8F04037
:10732C0002F046B90120DFE7FD70000008B5F9F75F
:10733C00D7FE002008BD012809D84FF08042D2F8B2
:10734C00783503F0010383F00103C2F878357047F8
:10735C00034640B1426802F00302022A06D0032A17
:10736C0004D0012A05D06FF0150070471A68002A66
:10737C00F9D0002098607047426802F00302022A9C
:10738C0010B5034681600AD0032A0BD10468002093
:10739C0000225A6008B1FFF74BFE204610BD006872
:1073AC000024F5E700242046F2E7002070470FB4D4
:1073BC0007B504A951F8040B0191F9F7EDFE03B0E0
:1073CC005DF804EB04B07047038B13F0070305D191
:1073DC000368002B0CBF002003207047022B05D143
:1073EC00438B002B14BF002004207047012B05D1C8
:1073FC000368002B0CBF002005207047002070474D
:10740C002DE9F0410D4607461946281D90461E46AB
:10741C00FFF7B2FF044638B1334642462946384698
:10742C00A446BDE8F0416047BDE8F08110B44FF0D0
:10743C002004EFF3118284F31288BFF36F8F416144
:10744C0010BC0121F9F7B6BE10B50C4640B139B1EC
:10745C00081DFFF77DFF28B9A36833F0030301D0A3
:10746C006FF0150010BD38B50C46054658B151B13A
:10747C000B6843B14B6833B11C22002101F090FC26
:10748C002C61002038BD6FF01500FBE770B5044689
:10749C000E46FFF7D9FF051E31DB4FF02003EFF34B
:1074AC00118183F31288BFF36F8F638B208B4FF6A0
:1074BC00FF75AB4200F007022ED0022A0ED1013329
:1074CC0063831546012381F31188BFF36F8FB3B12A
:1074DC00002331462046FFF793FF10E0830701D0CD
:1074EC00062A0ED100233360636893B9C4E90066A1
:1074FC00154662B90A4620460221F9F75BFE28467A
:10750C0070BD052A0CBF6FF085056FF004050023D4
:10751C00D9E71E606660EBE76FF00A05F7E70446F3
:10752C0008B5084611461A46A047FFF765FBFCF75D
:10753C008DFD00EBC100408840087047F8B503464C
:10754C00FFF7F7FFB0FA80F0C0F11F0003EB800CDF
:10755C00CA00DCF81060171D0C4606328DB256B905
:10756C00012101FA00F0D9680143D960CCF8104030
:10757C00DD539D52F8BDF1000431585AD85303EB3A
:10758C00C0009E52C5805D52F4E7043ACB1D1144F5
:10759C0023F0070321F00701F0B4CD1AEA080360C9
:1075AC00B2FA82F0C0F12404A40007340026E108EA
:1075BC00C0F1200003F110049A60DE6004EB80003F
:1075CC00844218D1480040F00100588003EBC104FC
:1075DC00501A47001E8067805C1923F8311003EBAA
:1075EC00C20266805853508840F001005080F0BCB5
:1075FC001846FFF7A3BF44F8046BE1E72DE9F84FF9
:10760C009A46D3786F2B80460F461546A3F1410B53
:10761C0029D024D8582B14BF0A261026DDF8289020
:10762C003246002340463946F8F752FD092AD4B2B7
:10763C001ED83034B045E4B277F1000309F8014D9F
:10764C0001D3D14511D82B789B0605D5082E15D121
:10765C00AB7843F00803AB704846BDE8F88F03F0F5
:10766C00F703702BD7E70826D8E780460F46D7E7F5
:10767C00BBF1190F94BF37345734DBE7102EEBD125
:10768C00AB7843F01003E6E72DE9F0410746884656
:10769C0015461E461446B442A4EB050002D33EB96F
:1076AC0023782BB114F8010B4146B8470028F2DAC5
:1076BC00BDE8F081F0B54668C7684569C369A6EBBB
:1076CC00070C751B63450446A3EB05009CBFACEB94
:1076DC00030CFF18824228BF0246A3EB0C00904219
:1076EC00236828BF1046F71B1F4406440F606660D2
:1076FC00F0BDD0E90123D21A8A420BD31944C368D6
:10770C00C269C0E90111C91A8A4201D81344C36085
:10771C00002070476FF0150070472DE9F34180464B
:10772C000E46154600272A4601A94046FFF7C2FF20
:10773C00314604460246019801F027FB2D1B2744D5
:10774C00264401D0002CEED139464046FFF7D1FF3C
:10775C00384602B0BDE8F081F0B586690569C369A9
:10776C008768A5EB060C63450446A7EB05009CBF98
:10777C00ACEB030CF618904228BF10460746A3EB5F
:10778C000C00B842236828BF3846AE1B1E44054483
:10779C000E602561F0BDD0E90423D21A8A420BD3C6
:1077AC001944D0E90632C0E90411C91A8A4201D839
:1077BC0013448361002070476FF0150070472DE96A
:1077CC00F34180460D4616460027324601A9404635
:1077DC00FFF7C2FF04462DB102460199284601F07D
:1077EC00D4FA2544361B274401D0002CEDD1394660
:1077FC004046FFF7D0FF384602B0BDE8F0810B07DA
:10780C0004D5A0F14103192B98BF203070472DE906
:10781C00F04F87B08A4614460293054618B90120EA
:10782C0007B0BDE8F08F0029F9D0029B002B00F0C7
:10783C00138104F004030A460493A946214619F85F
:10784C00010BFFF7DCFF0346C0B23F281778064652
:10785C0025D013F0C00F0BD1C8B12A2836D0214641
:10786C003846FFF7CCFF864202F101021ED0D6E764
:10787C005B287BD05C28F2D1E007F0D46878FFF766
:10788C00BEFF10F0FF0618BF05F10209E7E7E3069B
:10789C0001D52F2FC4D0381E18BF0120C0E7002FF0
:1078AC00BDD02F2F04D1A607B9D401324D46C4E761
:1078BC002E2FFAD1049B002BF7D05245AFD0A50741
:1078CC00F3D512F8013C2F2BEFD1A8E76878FFF71E
:1078DC0096FFC1B22A2918D02E2F09D1049B3BB197
:1078EC0052459CD0A00703D512F8013C2F2B96D003
:1078FC0079B914F0020093D0E30600F1AF802F2188
:10790C00104601F0DEF90038C6E719F8010F2146E0
:10791C00DDE72F2921D0029B16465F1E24F00408B8
:10792C0004F0020AB34621469BF80000FFF767FFFC
:10793C0010F0FF0506F101063FF471AF3B464246DD
:10794C0059464846FFF763FF01287FF469AF2F2D96
:10795C00E8D1BAF1000FE5D061E7A707DBD51046F7
:10796C0001F0AFF902460028A0D158E7002F3FF4F0
:10797C0056AF2F2F02D1A6073FF551AF21463846FF
:10798C00FFF73DFF6B780090212B01D05E2B23D1AC
:10799C00023501230193012304EA03014FF0000B8C
:1079AC0003912E46214616F8010B0593FFF727FF8E
:1079BC005FFA80F8B8F15D0F059B10D10BBB019BF2
:1079CC005B453FF42CAF731C03D15B2F7FF427AFC7
:1079DC004E460132B14669E74D460023DAE7B8F16D
:1079EC002F0FF2D0B8F15C0F07D1039B4BB968781D
:1079FC00FFF705FFAE1C5FFA80F8B8F1000F3FF4FB
:107A0C000EAF33782D2B20D170782146FFF7F7FE7F
:107A1C0010F0FF0019D05D2817D05C2806F1020584
:107A2C000AD1039B43B9B078FFF7E9FE10F0FF00D1
:107A3C0006F103053FF4F3AE009B434503DB8342A1
:107A4C00D8BF4FF0010B0023ABE7009B35464345F5
:107A5C0008BF4FF0010BF6E70320E1E60846DFE62E
:107A6C004023FFF7D4BE704708B50020FAF744F85E
:107A7C0008B50120FAF740F883681B6A03B1184770
:107A8C00704743681B6810B51C682046FFF7F4FF6D
:107A9C00A368DB6A0BB120469847002010BD08B5DF
:107AAC0043681B68197411B11868FFF7E5FF0020D3
:107ABC0008BD10B51C464368D868FFF780FE2060EF
:107ACC00002010BD2DE9F04145681E462B681B7C3B
:107ADC000C46174653B101EB020844452B6820D1E4
:107AEC00D3E9012137600120904717E0A868FFF720
:107AFC0014FE2B6830600C330121BFF35B8F53E80D
:107B0C00002F43E800100028F9D1BFF35B8F2AB98E
:107B1C002B6818688368DB6903B198470020BDE8BF
:107B2C00F081186814F8011B83685B689847D4E7E8
:107B3C002DE9F34180460D4683685B6C03B1984791
:107B4C00D8F808305B6B0BBB0027E86801A9C26949
:107B5C00FFF7B0FDD8F80830064678B39B69019959
:107B6C004BB30246404698470446002CE868214631
:107B7C0018BF0127FFF7BDFD0CB1A642E5D04FB1F0
:107B8C002B680020D3E90121904703E04046984739
:107B9C000028D9D1D8F808305B6ADBB9A86801A9EC
:107BAC00C269FFF7D9FD0446D8B94046FFF764FF18
:107BBC002B68DC6021E06FF05704D6E79B6933B18A
:107BCC0001220DF10301404698470446D4E76FF0BB
:107BDC005704D1E7404698470028DFD102B0BDE8F2
:107BEC00F081D8F8083001995B6963B102464046D0
:107BFC0098470146A868FFF7CEFD2B680120D3E912
:107C0C0001219047EAE76FF05701F3E70346BFF312
:107C1C005B8F53E8000F40EA010243E8002CBCF1F3
:107C2C00000FF6D1BFF35B8F70470346BFF35B8F3A
:107C3C0053E8000F00EA010243E8002CBCF1000FEE
:107C4C00F6D1BFF35B8F704773B58568090101F5F9
:107C5C001A71044616460D4401AA6946284601F0DD
:107C6C004BFF009B23B1284601F043FF2046B04751
:107C7C0002B070BD08B510B101F031F880B208BD8A
:107C8C000EB403B503AA52F8041B0192FBF7B0F92A
:107C9C0002B05DF804EB03B07047FEF7B1BB8B6824
:107CAC0020B903F51A700021FFF7C2B903F526704D
:107CBC00F9E738B58368D3F86432DB0704461AD485
:107CCC00406803685B689847054620B9E06800F097
:107CDC00CDFDA3681D71A3685B6B13B129462046CB
:107CEC009847A3680022C3F80C23FEF785FFBDE874
:107CFC003840FCF7ABB96FF00F05ECE700F51970E5
:107D0C0011B10421FFF782BF6FF00401FFF78DBFA3
:107D1C0008B500F5187029B10121FFF777FF00F0C5
:107D2C00010008BD6FF00101FFF77FFFF7E7FEF7D9
:107D3C00DFBBF8B5044680681F460379022B0D465D
:107D4C00164607D0BDE8F8404FF4805100F5197085
:107D5C00FFF75CBF4FF0FF324FF0FF3300F53E7082
:107D6C00FFF79BFFA368D3F86422110504D49B6B27
:107D7C0013B9204600F04CFB3B46324629462046C0
:107D8C0000F0A7FBA368D3F86422120504D49B6B04
:107D9C0013B92046FBF7B6FA606900F044F8A06806
:107DAC00BDE8F84000F53E70FFF7C1BF0CB407B555
:107DBC0004AB53F8042B0193FFF7BBFF03B05DF842
:107DCC0004EB02B070472DE9F04107460E4614460D
:107DDC000D460CB9BDE8F081102CA04628BF4FF021
:107DEC0010082A46A91B43463846FBF799F8A4EB22
:107DFC0008044544EDE710B5044680684FF0FF32A7
:107E0C004FF0FF3300F53E70FFF747FF2046FAF7BF
:107E1C0043FAA068BDE8104000F53E70FFF787BF3D
:107E2C00836899637047026983681268016810B5AA
:107E3C000446C0689847236900221A6010BD38B503
:107E4C00CB681B7C022B05460C4604D10A2802D1B8
:107E5C000D20FFF7F4FF236922681B68D5542269B3
:107E6C001368013313606268934202D12046FFF716
:107E7C00DAFF002038BD202805D0093804288CBF33
:107E8C000020012070470120704708B510B100F0A8
:107E9C0026FF80B208BD10B5037B40891A441944F3
:107EAC00B2FBF0F4B1FBF0F300FB142200FB131057
:107EBC00101A10BD10B5047B438921441019B1FB75
:107ECC00F3F1B0FBF3F0401A10BD30B5057B4389DC
:107EDC002944B1FBF3F403FB141101312A4401349E
:107EEC000180B2FBF3F103FB1122848001324C1CA4
:107EFC00C480428030BD2DE9F84F002506460F4660
:107F0C001446984605602078002800F0B580FFF7ED
:107F1C00B2FF18B1002304F8013BF4E73268531C9C
:107F2C004345336047F8224000F0A680054694F89C
:107F3C000090B9F1000FE6D0002D40F08980B9F126
:107F4C00270F06D0B9F15C0F00F08A80B9F1220F2F
:107F5C0076D12046FFF799FF611C0246204600F0BF
:107F6C00FCFE4D46E3E72046FFF78FFF611C0246FF
:107F7C00204600F0F2FE0025D9E7302926D1022355
:107F8C004FF0000AE15CA1F13002D2B2072A5FFA8D
:107F9C0083F918D8013342EACA0A052B5FFA8AFA28
:107FAC00F0D199462046FFF770FF09F1FF3BA3443F
:107FBC00A9F10209A0EB09025946204600F0CDFEBA
:107FCC0004F801ABB3E7B9F1020FEBD178293DD13D
:107FDC0002214FF00009625CA2F13003DBB2092BE5
:107FEC00C8B21AD843EA091203295FFA82F912D1EE
:107FFC004FF0040A2046FFF748FF0AF1FF3BA34469
:10800C00AAF1020AA0EB0A025946204600F0A5FE8E
:10801C0004F8019B8BE70321DDE7A2F16103052B3B
:10802C0003D8573A42EA0912DEE7A2F14103052BC5
:10803C0001D8373AF6E7022808D04FF0030AD9E7FF
:10804C004846FFF718FF00287FF45DAF01346EE758
:10805C00A94588D0B9F15C0FF8D161788D428CD1EB
:10806C002046FFF712FF04F101090246494620465B
:10807C0000F073FE4C465AE72846BDE8F88FF8B579
:10808C000E4611461546074600F0DFFD044628460D
:10809C00FFF7FBFE0546C4B1A74207D214F8013C1A
:1080AC00202B02BF0135ADB204F1FF342046FFF79F
:1080BC00ECFE3388421C5B1B521B3380611920463B
:1080CC0092B2BDE8F84000F048BEF8BD2DE9F04191
:1080DC00884686B01746044628B10146142201A8EA
:1080EC0000F053FE01AC002631463A462046FAF722
:1080FC0093FF0136054628B12968404600F0FFFD84
:10810C000028F1D1284606B0BDE8F0812DE9F047F2
:10811C001C46DDF820809DF8249000230F4616465F
:10812C0023602368BB4205461BD256F8230000F09F
:10813C0016FC2368824618B1013323602846F0E709
:10814C0056F8231042462846FFF7C0FF48B1236873
:10815C005A1C2260B9F1000FE3D08045E1D12360B5
:10816C0055462846BDE8F0872DE9F0410746FFF754
:10817C008CFE064647BBBDE8F0814CB192B2B21AF8
:10818C00581C0132384400F0E8FD361BB6B24446A8
:10819C00731E9D42EFDA785DFFF76DFE2B460135BD
:1081AC00ADB20028F4D02A4691B28E42F0D9B85C18
:1081BC00FFF761FEB91802F1010C80460028DCD0F3
:1081CC000134A4B26246EFE700252C46E0E7F8B58F
:1081DC00846894F84230054653B9AB689A8FDA87B5
:1081EC00F8BD013A92B2A28722B984F84220F4E792
:1081FC0004F14206A28FB31813F8010CFFF73BFEF3
:10820C0003460028EDD1B0549FB216FA83F1F05D0D
:10821C00FFF731FE01330028F6D1002FDDD0A38FFC
:10822C000133DA1B304600F098FDA38FDB1BA387CC
:10823C00D3E70EB403B503AA52F8041B0192FAF764
:10824C00D7FE02B05DF804EB03B07047826838B516
:10825C0004461068958F10B100F041FD80B2A26801
:10826C004319508DB3FBF0F200FB1230B0FA80F0E2
:10827C00400938BD826838B504461068D58F10B1F6
:10828C0000F02DFD80B2A2684319508DB3FBF0F2C3
:10829C0000FB1230B0FA80F0400938BD10B504462E
:1082AC00FFF7E8FF20B16069BDE81040FAF7E6BEC1
:1082BC002046FFF7CBFF0028F5D110BDF8B5846838
:1082CC000546A28FE18F04F12000FFF7FEFD284642
:1082DC00A78CE68CFFF7BAFF10B16869FAF7CEFEEF
:1082EC00B74207D1218C638C2846C91ABDE8F840E7
:1082FC00FAF7E0BEE18CA38C2846C91AFAF7C4FE43
:10830C00F0E7F8B5044680680D46C18F828F2030A7
:10831C000D44FFF7DAFDA068ADB2C18F2A462030BC
:10832C00FFF7C8FD0746A0682A46C18F2030FFF72B
:10833C00B2FD794206462046FAF7A6FE31462046A3
:10834C00FAF7B8FEA368DD87F8BD2DE9F8430C1EDB
:10835C00064634DA644224B24FF0FF35A4B2AFB211
:10836C0025E0B368B3F83EE0B3F83C9003F1420863
:10837C0000207346A3EB0E0189B20BB96A1C10D016
:10838C00994501D1012D0CD018F8032042F0200C96
:10839C00ACF1610CBCF1190F0DD9303A092A0AD98C
:1083AC0050B109B23046FFF7ACFF013CA4B2002C2F
:1083BC00D7D1BDE8F88301203B449BB2DAE7012515
:1083CC00CCE78368D98F494209B2FFF79ABF83681B
:1083DC00998FDB8FC91A09B2FFF793BF8368DB8FC4
:1083EC001BB14FF0FF31FFF78CBF70478368DA8FFA
:1083FC009B8F9A4202D20121FFF783BF704783689B
:10840C00DA8F9A871344002283F84220FAF72ABEA7
:10841C0010B504468068828FC18F2030FFF755FD60
:10842C00A368198C2046C1F10101FAF743FEA36839
:10843C00998C20460139FAF727FE2046BDE81040FA
:10844C00FAF710BE2DE9F041054686B00F461446EA
:10845C00002614B906B0BDE8F081686803682246AE
:10846C00D3F80C80B9196B46C047009A1644A41A6D
:10847C00002AEED1AB6819790329EAD0022913D866
:10848C0003F52673012101A801F011FB4FF0FF3217
:10849C004FF0FF33012101A8FEF76EFDA86800F52F
:1084AC00267001F026FBD4E7D3F864229207FBD5A3
:1084BC00BFF35B8F03F5197353E8002F22F0020210
:1084CC0043E800210029F7D1BFF35B8FC1E7FFF729
:1084DC00B9BFF7B50F4681681E46D1F86032DB068E
:1084EC000446154617D591F82E30BB4213D0022204
:1084FC002E3101A800F049FC39462046FAF7F8FD68
:10850C00606932462946FAF773FD01A92046FAF74D
:10851C000FFE03B0F0BD60693246294603B0BDE8DA
:10852C00F040FAF765BD0CB407B504AB53F8042B57
:10853C000193FFF7CEFF03B05DF804EB02B0704778
:10854C002DE9F0418668B58FAB18FF2B074688469E
:10855C0014461EDCF38FED1A42331E44ADB22A468C
:10856C003146301900F0F9FB22464146304600F006
:10857C000CFCB9688B8F23449BB28B870B44002275
:10858C0083F84220D1F860329B0704D4CA8F14447C
:10859C00CC87BDE8F08129463846BDE8F041FAF7B2
:1085AC0041BEFFF7CDBF38B5836805469C8FD88F89
:1085BC00241AA4B28CB1423018442246411C00F05B
:1085CC00CCFBAA68938F611E013B9387284601223E
:1085DC00BDE8384089B2FAF725BE38BD83689A8F5A
:1085EC0010B5044652B1DB8F43B14FF0FF31FFF7AA
:1085FC0088FE2046BDE81040FFF7D5BF10BD0EB475
:10860C0003B503AA52F8041B0192FAF7F1FC02B06D
:10861C005DF804EB03B070472DE9F0470446904633
:10862C000E46002969D00025735D202B23D0093B11
:10863C00042B20D9304600F052FBA368598D80B230
:10864C00401BA1EB0803984206EB050915D94846D7
:10865C00002710F8012B202A06D0A2F1090CBCF13E
:10866C00040F02D80A2A2FD03B4608EB070291428E
:10867C0029D90137EDE70135D6E74B460027B8423B
:10868C0016D013F8012B0A2A05EB070A19D16069D9
:10869C00FFF7C9FB49463A462046FFF7D3FE60690F
:1086AC00FAF748FE414620460AF10105FAF702FDA9
:1086BC0060697119FFF7A3FF6069BDE8F047FAF72D
:1086CC0039BE0137DBE71F466069FFF7ACFB3A4662
:1086DC0049462046FFF7B6FE3D44735D202B0AD079
:1086EC00093B042B07D96069FAF724FE4146204662
:1086FC00FAF7E0FC9EE70135EFE7BDE8F087836908
:10870C000020186070470EB403B503AA52F8041B7E
:10871C000192FAF76DFC02B05DF804EB03B0704700
:10872C008368BFF35B8F03F5187353E8002F22F0B7
:10873C00080243E800210029F7D1BFF35B8F00202A
:10874C0070478368BFF35B8F03F5187353E8002FF2
:10875C0042F0080243E800210029F7D1BFF35B8FF8
:10876C00002070478368BFF35B8F03F5187353E8E1
:10877C00002F22F0020243E800210029F7D1BFF3B9
:10878C005B8F002070478368BFF35B8F03F5187312
:10879C0053E8002F22F0100243E800210029F7D102
:1087AC00BFF35B8F002070478368BFF35B8F03F5CB
:1087BC00187353E8002F42F0100243E800210029FF
:1087CC00F7D1BFF35B8F002070478368BFF35B8FDB
:1087DC0003F5187353E8002F42F0020243E800211E
:1087EC000029F7D1BFF35B8F0020704708B5836871
:1087FC000068D3E900210A6051600021C3E900112F
:10880C001A895B891A440C32FEF7D9FF012008BD86
:10881C000023C3607047F8B51F460346164653F84D
:10882C00044F9C4202D100203880F8BDC568B1B914
:10883C00002DF8D0AC4202D10023C360F3E76C6882
:10884C00C460002CEFD0228904F10C01304600F0FA
:10885C009CFA23893B800022F2540120E5E7002D8D
:10886C00EED08368AB42E7D02C68E9E738B5044614
:10887C00051D6368AB4204D02046FFF7B7FF002804
:10888C00F7D138BD2DE9F04F036802F10C05C5F1A5
:10889C000009DB6909F0030985B04D449D4204468B
:1088AC000191174610D80023C3606AB1466800F1E5
:1088BC00040AB2450BD05EB13389934208D106F15C
:1088CC000C0000F039FA18B905B0BDE8F08F1E465F
:1088DC004FF000082068026983689A4201BFC0E922
:1088EC000288C0E90588C0F80480C0F810802A46C8
:1088FC0003A9FEF7DFFE854283461ED920682A466F
:10890C0003A9FEF7D7FE854218D172895A447281A9
:10891C00AB44039D01992F813A46A5F80A9005F1C5
:10892C000C0000F032FA62682068C5E9002A59464A
:10893C0055606560FEF7DDFEC6E7EAD020680021D1
:10894C00FEF7D7FE63689A45C4D02046FFF74EFF6A
:10895C00C0E7031DC0E901330023C360704710B5A5
:10896C00044608B9002010BD00F0B9F9002380B20C
:10897C008342F7D2E25C3F2A03D02A2A01D001338A
:10898C00F6E70120EFE710B5044680684FF48072DB
:10899C00002100F5A17000F003FAA068828F00F1AD
:1089AC00420100F5A17000F0F0F9A06800F5A1708B
:1089BC00FFF7DAFBA06800F5A17000F090F9A3684E
:1089CC000130A3F8400010BD10B504468068B0F823
:1089DC00402000F5A171423000F0D7F9A368B3F83C
:1089EC0040209A8710BD00F0BCBD0146006800F025
:1089FC00B8BD013140B2FBF785B800210120FFF76B
:108A0C00F2BF38B504460D4611461A46FBF752F82C
:108A1C0060B2691CFBF776F8204638BD08B5FBF749
:108A2C00A3F8BDE80840FBF781B910B50278202AFD
:108A3C00034600F10100F9D0A2F109010429F5D98E
:108A4C002B2A08D02D2A0ABF034600210121013B05
:108A5C0000200A2404E003460021F8E76043801A52
:108A6C0013F8012F303A092AF8D901B9404210BD48
:108A7C002DE9F843844688460446214614F8013B08
:108A8C00202BFAD0A3F109000428F6D92D2B2DD1D7
:108A9C004B788C1C0121002A5AD0102A09D1302B7A
:108AAC0007D1237803F0DF03582B4CD163781022C5
:108ABC00023401F10047013F0026B7FBF2FE3046BD
:108ACC0002FB1E79A3F13005092D15D82B469A42CD
:108ADC0022DD751C07D070451BD801D14B4518DC25
:108AEC0000FB0230012614F8013BEBE72B2B04BFF3
:108AFC004B788C1C0021CEE743F02005613D192DED
:108B0C000AD8A3F141051A2D34BF372557255B1B15
:108B1C00DDE74FF0FF36E6E7731C09D1FDF70CFAE1
:108B2C00222303603846B8F1000F07D1BDE8F88363
:108B3C0001B14042B8F1000FF8D00EB104F1FF3C86
:108B4C00C8F800C0F2E73023002AB2D10822B0E7FF
:108B5C00302BA6D00A22ACE72DE9F0410746884617
:108B6C000446214614F8013B202BFAD0A3F109004E
:108B7C000428F6D92D2B2FD14B788C1C4FF0010CDF
:108B8C00002A5ED0102A09D1302B07D1237803F0AC
:108B9C00DF03582B50D16378102202344FF0FF3191
:108BAC000026B1FBF2F102FB01FE6FEA0E0E30461D
:108BBC00A3F13005092D16D82B469A4223DD002E41
:108BCC001EDB88421CD801D1734519DC00FB023036
:108BDC00012614F8013BEBE72B2B04BF4B788C1CC4
:108BEC004FF0000CCCE743F02005613D192D0AD85D
:108BFC00A3F141051A2D34BF372557255B1BDCE744
:108C0C004FF0FF36E5E7002E0ADAFDF795F922233F
:108C1C0003604FF0FF30B8F1000F09D1BDE8F081CF
:108C2C00BCF1000F00D04042B8F1000FF6D006B1F5
:108C3C00671EC8F80070F1E73023002AAED1082275
:108C4C00ACE7302BA2D00A22A8E72DE9F04191F82D
:108C5C0000800546B8F1000F10D04C1C204600F0E7
:108C6C003EF807462E4616F8013B63B1984508D1ED
:108C7C003A462146304600F04EF810B92846BDE879
:108C8C00F0813546EEE71D46F8E70139034611F849
:108C9C00012F0AB91A70704703F8012BF7E770B56A
:108CAC0005462B4642B111F8014B561E2CB92A44ED
:108CBC0003F8014B9A42FBD170BD05F8014B3246CB
:108CCC00EFE7C9B203461A788A42184603F101034A
:108CDC0004D0002AF7D1002918BF002070470346A2
:108CEC0000201A5C02B970470130FAE703460020F5
:108CFC001A5C0AB1884200D170470130F8E7431E74
:108D0C00013913F8012F11F8010F824201D1002A09
:108D1C00F7D1101A704710B501390244824209D0BC
:108D2C00037811F8014FA34200D10BB9181B02E0D4
:108D3C000130F3E7002010BD10B503465AB10139DC
:108D4C00841813F8010B11F8012FA34201D09042A3
:108D5C00F7D0801A10BD1046FCE7431A934210B5A9
:108D6C0000EB020308D3013902469A4207D011F8EE
:108D7C00014F02F8014BF8E70A448A4200D110BDBA
:108D8C0012F8014D03F8014DF7E710B5431E0A44E4
:108D9C00914200D110BD11F8014B03F8014FF7E7D8
:108DAC00C9B202440346934200D1704703F8011B39
:108DBC00F9E74FF0FF3070474B68012B07DD0B686C
:108DCC0018700B6801330B604B68013B4B60002043
:108DDC007047062808D14FF080430122C3F80025C4
:108DEC00BFF34F8F20BFFDE77047002383F311883B
:108DFC00BFF36F8F70470369C9B20C2201FB0233BA
:108E0C00186C00F0070070474FF02003EFF311824D
:108E1C0083F31288BFF36F8F036803F0C00343F032
:108E2C000203036082F31188BFF36F8F7047034610
:108E3C0070B50069C9B24FF02004EFF3118684F3CA
:108E4C001288BFF36F8F0C2505FB0104246C14F002
:108E5C00C00401D0A24210D105FB01000122026422
:108E6C00002086F31188BFF36F8F28B95B6803EB82
:108E7C00C1014B689847002070BD4FF0FF30F0E700
:108E8C008022FFF7D4BFF8B5069F04690546C9B226
:108E9C004FF02000EFF3118C80F31288BFF36F8F2B
:108EAC000C2606FB0146306C00F0070EBEF1010FDC
:108EBC0011D1376400268CF31188BFF36F8F46B93C
:108ECC000C2000FB0144C4E90E236B6853F83130CD
:108EDC0098473046F8BD00F0C000874214BF4FF0F1
:108EEC00FF366FF07706E6E713B580240094FFF7A2
:108EFC00CAFF02B010BD006910B4CBB21C2403FB36
:108F0C000400002110BC1047002000F0C1BA10462C
:108F1C00FDF732BB83685B68184743685B68D3F81E
:108F2C0010350B600020704743685B68D3F804056C
:108F3C0042400A404240C3F8042500207047436871
:108F4C005B680020C3F80815704743685B68002015
:108F5C00C3F80C15704743685A68D2F804354B4077
:108F6C00C2F80435002070470369586830B558B111
:108F7C000024814212D108689D6854B98D42586012
:108F8C0000D19860002008606AB9002030BD2846E6
:108F9C00EFE78D42206008BF9C60F3E7056804464C
:108FAC00002DF4D13AB198685A680A6059600028CB
:108FBC00EBD19960EAE76FF01500E7E702690B4621
:108FCC00D2E9010183E803000020704743681B6865
:108FDC00D3F88004C3F880047047436802691B68A7
:108FEC00D3F8100148B1527D0A700020C3F810016B
:108FFC00D3F8102101221A6070474FF0FF307047F0
:10900C00002A10B504460FDD43681B68D3F8100125
:10901C0048B122690020C3F81001D3F81001527D29
:10902C000A700120186010BD0020FCE7436801693C
:10903C001A684FF02000EFF3118380F31288BFF30E
:10904C006F8FC968002088734FF48001C2F8041335
:10905C0083F31188BFF36F8F70470369DB680122BC
:10906C009A7370470369DB689A7B02F0FF0162B95F
:10907C0042681268D2F8580140B1D2F8040310F4D7
:10908C00800003D0196101207047002070474368AD
:10909C001B68D3F81001003818BF012070474368D3
:1090AC001B681022C3F80423704743681B68102206
:1090BC00C3F80823704743681B684FF40072C3F869
:1090CC000423704743681B684FF40072C3F80823ED
:1090DC007047012070470369DB68C3E900127047D1
:1090EC0038B543681D68D5F804335B02044605D4D3
:1090FC00D5F8040310F0100006D138BDFFF7B2FF0D
:10910C000028F5D00120F8E72046FFF7C0FF003813
:10911C0018BF0120F1E70368C3F84415C3F84825CC
:10912C000022C3F82021D3F82011C3F85821D3F81A
:10913C0058214268D20641BF0822C3F800254FF4DB
:10914C008002C3F8042301229A6070470268034628
:10915C00D2F8580140B95B689B0706D4D2F82001BD
:10916C00003818BF0120704701207047F8B5066918
:10917C00F3689C89BFF35B8F9442A8BF14460546E5
:10918C001033012253E8000F002803D143E80027D5
:10919C00002FF7D1BFF35B8F0CBF134600231DD0FC
:1091AC001C462046F8BDF268C85C9268D054013366
:1091BC00A342F8DB4FF02003EFF3118783F31288FF
:1091CC00BFF36F8F6868FFF7C1FFF36840B9186190
:1091DC00044687F31188BFF36F8FE2E70023E7E7BC
:1091EC00996868682246FFF796FFF2E742681368B1
:1091FC00D3F80413C90510B418D5D3F82011A9B1AC
:10920C004FF02004EFF3118184F31288BFF36F8FBA
:10921C00D3F8204134B10024C3F82041D3F82041C5
:10922C000124DC6081F31188BFF36F8F5268D20682
:10923C001AD54FF02002EFF3118182F31288BFF39D
:10924C006F8FD3F8582112B10022C3F800250269A0
:10925C00D2680AB112691AB94FF48002C3F8082314
:10926C0081F31188BFF36F8F0269D2685AB1D3F8BA
:10927C00581151B1947B0021116134B14FF480002D
:10928C00C3F80803917310BC7047D3F8241121B1B3
:10929C000021C3F82411D3F824311368002BF2D029
:1092AC00516810BC1847704708B5FBF7AFFD08BDF7
:1092BC0030B543681360037A03F10053013BDB00C4
:1092CC00456814681D44AC4202D96FF0010030BDF2
:1092DC0065798D4202D008341460F1E70020F6E77E
:1092EC0000F01F03012098404FF0A04311B9C3F8C0
:1092FC000C057047C3F80805704700F48053002B29
:10930C0010B500F01F0308BF1446C0F3811200F41F
:10931C00706018BF002140EA820242EA010218BFC5
:10932C00012403F5E0734FF0A04142EA440241F8F6
:10933C00232010BD2DE9F0411446804600EB810737
:10934C0001254FF0A046B84502D10020BDE8F081C0
:10935C00D8F800301A0C192A75D8DFE802F00D1B6A
:10936C002249273C49747474744E53747474747425
:10937C007474747458656A6F03F03F03C4F80C3549
:10938C00D8F8003003F01F0305FA03F3C6F80835CC
:10939C00012204E003F03F03C4F814350022114607
:1093AC0012E003F03F03C4F80835E9E703F03F038C
:1093BC00C4F80835D8F8003003F01F0305FA03F39E
:1093CC00C6F80C3500220121D8F80000FFF795FFF4
:1093DC0008F10408B7E703F03F03C4F80C35D8F8DC
:1093EC00003003F01F0305FA03F3C6F80C35CFE782
:1093FC0003F03F03C4F81035D0E703F03F03C4F883
:10940C000835CBE703F03F03C4F80C35C6E703F08F
:10941C003F03C4F86035D8F80000C0F3403100F0C9
:10942C003F00FFF75DFFB3E703F03F03C4F864357B
:10943C00F1E703F03F03C4F86835ECE703F03F03B2
:10944C00C4F86C35E7E76FF085007FE708B50020BE
:10945C00FAF710FF4FF08053D3F83001421C04BFD1
:10946C004FF0704393F8E00F831F584258417047F8
:10947C00004700F0E9B908B50020FAF767FB08B916
:10948C00FAF754FB4FF080430022C3F8182508BDAF
:10949C00FCF71CB800F01F00800000F1A040D0F8D1
:1094AC00003723F4403343EA0143C0F800377047D8
:1094BC0003680122DA60704730B54FF480340068DD
:1094CC008C4063B18B0003F5A0730025C550C358C5
:1094DC00C0F8044301F5A87140F8212030BDC0F854
:1094EC000843F7E770B4046840F20116D4F8005250
:1094FC008E4025EA0605C4F80052D4F800522B43DE
:10950C00C4F800329DF80C3070BCFFF7D5BFFCF7E7
:10951C0081BC08B5FFF7FBFF002008BD704738B1D0
:10952C00C3681888C0F30800A0F5807358425841EE
:10953C007047406970B413460D4660B901462A461F
:10954C0070BCFCF79DBC013130F811403444A4B21E
:10955C009442F8D9F3E7002147F6FF764FF6FD72F7
:10956C00F2E7F8B505460E464FF02003EFF31187EE
:10957C0083F31288BFF36F8FFDF73EFB3146044631
:10958C002846FFF763FF87F31188BFF36F8F2046E0
:10959C00BDE8F840FAF75ABDFFF702BCFFF7F5BB80
:1095AC00EFF30580003818BF012070477830704702
:1095BC00FDF76EB910B500238B4202D11360002069
:1095CC0010BDC45CAA2CF9D10133F5E70A46D0E9E9
:1095DC002701FFF7EFBF08B5FAF754F9BDE80840CB
:1095EC00FFF761BE90F90E308B4201D0FDF7C0B988
:1095FC000020704703460020C3E90200C3E9003392
:10960C007047D0E9003213605A600023C0E9003380
:10961C00704708B5FFF7F5FF437B23F00203437354
:10962C000023836008BD90F90E3091F90E0083423F
:10963C0014BFC01A0020704710B54FF02003EFF391
:10964C00118483F31288BFF36F8FFFF7E2FF84F36B
:10965C001188BFF36F8FBDE81040183000F0AEB822
:10966C00034620B9EFF305820AB9FAF79DBA83F3E2
:10967C001188BFF36F8F70474FF02003EFF3118009
:10968C0083F31288BFF36F8FFFF7EABF03460068BE
:10969C00834208BF0020704710B54FF02003EFF352
:1096AC00118483F31288BFF36F8FFDF7BBF884F33B
:1096BC001188BFF36F8F10BD10B501464FF020031A
:1096CC00EFF3118483F31288BFF36F8F10F80B3C08
:1096DC0013F0280F0DD151F8103C18380BB1FFF7CF
:1096EC0098FF11F80B3C23F0140301F80B3CFDF729
:1096FC0099F884F31188BFF36F8F10BD38B5044609
:10970C000D46FDF7E3F8637B43F00203637395B1F9
:10971C002B68A5609D4215D0A3B194F90E1093F956
:10972C000E20914208D0521A002A05DD5A68C4E96D
:10973C00003214605C6038BD6A68934202D01B68CA
:10974C00002BECD16B68C4E900531C606C60F2E731
:10975C0038B54FF02003EFF3118583F31288BFF374
:10976C006F8FFFF793FF044620B1FFF752FF1830BD
:10977C0000F024F885F31188BFF36F8F204638BDB5
:10978C0038B54FF02003EFF3118583F31288BFF344
:10979C006F8FFFF77BFF044658B1C0F8B0104261E1
:1097AC00FFF737FF183000F009F82046FDF73AF8BC
:1097BC00012085F31188BFF36F8F38BD10B54FF0C2
:1097CC002002EFF3118482F31288BFF36F8F0368CA
:1097DC003BB1FDF7C9FA002084F31188BFF36F8FFA
:1097EC0010BD6FF01500F7E710B54FF02003EFF345
:1097FC00118483F31288BFF36F8FFDF78FFA84F314
:10980C001188BFF36F8F10BD70B504460D464FF035
:10981C002003EFF3118683F31288BFF36F8FFDF7EC
:10982C007DFA012805DDA04203DB29462046FBF723
:10983C0069FC86F31188BFF36F8F70BD08B5FDF717
:10984C0083FB08BDFDF780BB08B1FAF729BD704753
:10985C00F8B50D46D0E90013884204460DD063B12B
:10986C00986800B16038A2F160073946FFF7DBFE5B
:10987C00002802DC2668B44209D16368C5E90043BC
:10988C001D606560F8BD6368B342F6D03668002E83
:10989C00F3D0B16801B160393846FFF7C4FE002837
:1098AC00F1DD7368C5E900631D607560EAE72DE9B9
:1098BC00F84F00258B4614461F4682462E46A84676
:1098CC005D4502DB3046BDE8F88F4FF02003EFF327
:1098DC00118983F31288BFF36F8F9AF80D3003F060
:1098EC001F03013B072B0FD8DFE803F01E040E0A01
:1098FC000E0E0E25DAF810309B682BB1022320E0F7
:10990C00DAF810301B688BBB47BB237833B39AF85B
:10991C000D3003F01F03013B072B30D8DFE803F0B9
:10992C0033282F282F2F2F38DAF810309B68002B74
:10993C00EAD0012305E0DAF810301B6A002BE3D0E3
:10994C001023DAF80C20CAF80880C2F345310B4317
:10995C0063F35232CAF80C2084F8008089F3118822
:10996C00BFF36F8F01350AF1140AA9E70423E8E766
:10997C00DAF81000224651461030FFF769FFCAF89A
:10998C0008400136EAE7DAF8100022465146F4E7BF
:10999C00DAF81000224651462430EEE72DE9F84360
:1099AC00846805460E4644B16378012B36D114F811
:1099BC00533C13F002030AD12370EB68C3F3453117
:1099CC000E43002066F35233A860EB600BE054E9C1
:1099DC000E23B3F1FF3F08BF12F1020F05D1002394
:1099EC0023706FF00A00BDE8F883A4F160084046CC
:1099FC00FFF722FE082E0CBF6FF003030023236534
:109A0C0014F8533CDB0602D154F8487C0FB1002308
:109A1C00D2E74046FFF740FE2770CEE7022BF6D187
:109A2C002378002BC9D054F8047C002FF4D04FF0CD
:109A3C000008A4F1140904F11400FFF7BFFEC4F8E8
:109A4C002C804946384600F076F884F80080B4E75C
:109A5C001423F0B503FB01000024012601B9F0BD6D
:109A6C0010F8073C40F80C4C03F01F03082BA0F136
:109A7C0014070DD806FA03F313F48B7F08D050F8B3
:109A8C00143C2BB150F8105C2B605D6040E9054430
:109A9C0082F31188BFF36F8F4FF02003EFF3118225
:109AAC0083F31288BFF36F8F01393846D6E710B5B0
:109ABC00D204090201F4F85102F400220A43017B9A
:109ACC0000240A43C0E90323846010BD03460068E8
:109ADC00834208D0D0E9003213605A600023C0E9F9
:109AEC000033FFF75BBF70470023C0E900008360C1
:109AFC00704700238360704783680B60C3681360F2
:109B0C00704710B400F10C04C0E9034410BCFDF71D
:109B1C003CBD026801238B4022EA0303036022FA56
:109B2C0001F000F00100704720B100221146C03056
:109B3C00FFF726BE704737B5019008464FF020035B
:109B4C00EFF3118583F31288BFF36F8F01A9FDF733
:109B5C0065FB044685F31188BFF36F8F002809DD80
:109B6C004FF02003EFF3118083F31288BFF36F8F54
:109B7C00FFF776FD204603B030BD7047FBF71ABBEC
:089B8C008465FF7F0100000069
:109B9400514200000000000065430000EC9B0000FF
:109BA4001F95000000000000A570000000000000E8
:109BB40049480000049C0000654B00001C9C000008
:109BC4005147000000000000A54F00000000000005
:109BD4002122000000000000C97000000000000005
:089BE400C10B000000000000AD
:109BEC0040BF0000D0A40000B8A400007402002004
:109BFC005C090020349D000046BF000040A5000019
:109C0C001CA5000078020020B80900202E9D000041
:109C1C004DBF0000C0A5000074A500007C02002010
:089C2C00B0000020289D00009B
:109C3400A4B6000014000020F405002064000020F5
:109C4400020000003CA20000040900200000000003
:0C9C5400ADB6000080020020401100208E
:109C600000000000889D0000000000007CA20000B1
:109C7000000000009C9D00000000000078A1000092
:109C800000000000E4A1000000000000B09D000002
:109C90000000000068A200000000000090A2000088
:109CA000000000008CA0000000000000A4A4000040
:109CB00000000000C49D000000000000D89D0000CE
:109CC00000000000EC9D000000000000A4A20000C5
:109CD00000000000B8A2000000000000009E00008C
:109CE00000000000149E000000000000289E0000FC
:109CF000000000003C9E000000000000509E00009C
:109D000000000000649E000000000000789E00003B
:109D1000000000008C9E000000000000A09E0000DB
:089D200000000000B49E0000E9
:109D280000800080FF7F00800080FF7F008000802F
:029D3800FF7FAB
:069D3A00FFFFFFFFFFFF29
:109D40001B5B4A00001B5B4800001B5B324A0000A3
:109D50001B5B4A00001B5B6D00001B3700001B38BB
:109D600000001B5B3F336C00001B5B4800001B5B6B
:109D7000324A00001B3700001B38000000000000C2
:109D80000338FDD87047000098AD00009FAD00007B
:109D900000000000397300000000000076AD0000F4
:109DA00080AD00006CA000003D0C00000000000031
:109DB00004AE000010AE000000000000010800002A
:109DC00000000000EEAC0000FBAC000074A000003E
:109DD000CD0B0000000000001FAC000030AC000004
:109DE000000000005906000000000000B7AB0000B2
:109DF000C0AB000000000000150B000000000000D8
:109E000059AE000067AE000000000000A10700008E
:109E10000000000057AC000075AC0000000000001E
:109E20009D09000000000000D1AB0000DAAB00008B
:109E300000000000C50A00000000000001AC0000A6
:109E400010AC000000000000250A00000000000027
:109E500050AD000061AD000000000000C10800002E
:109E60000000000016AD000031AD00000000000051
:109E70001109000000000000E3AB0000F2AB00009D
:109E800000000000750A000000000000BFAD0000E7
:109E9000CFAD0000000000006108000000000000DD
:109EA0005DAB00006FAB000000000000590B00002C
:109EB00000000000C0AC0000D1AC00007CA000009D
:109EC000050C0000000000008AB0000094B0000003
:109ED00000000000B104000000000000BBB0000062
:109EE000C5B00000000000008D040000000000006C
:109EF000ECB00000F8B000000000000069040000B1
:109F00000000000021B100002BB1000000000000A3
:109F1000450400000000000049B1000053B10000FA
:109F2000000000002104000000000000000000000C
:109F30000000000000000000000000000000000021
:109F400087AF00008FAF000000000000D1050000C7
:109F500000000000A0AF0000A8AF0000000000005B
:109F6000B505000000000000B9AF0000C1AF00005F
:109F7000000000009905000000000000D1AF0000C3
:109F8000D9AF0000000000007D05000000000000C7
:109F9000EAAF0000F2AF0000000000006105000021
:109FA0000000000003B000000CB000000000000042
:109FB00045050000000000001EB0000027B00000B2
:109FC00000000000290500000000000039B000007A
:109FD00042B00000000000000D050000000000007D
:109FE00054B000005DB0000000000000F10400006B
:109FF000000000006FB0000078B00000000000001A
:10A00000D504000000000000000000000000000077
:10A01000000000000000000000000000DAAE0000B8
:10A02000E9AE00000000000035060000000000005E
:10A0300011AF000022AF0000000000001106000078
:10A04000000000004CAF00005DAF00000000000009
:10A05000ED0500000000000000000000000000000E
:10A0600000000000000000000000000000000000F0
:10A07000C89E000000000000409F0000000000009B
:10A080001CA0000000800040000400008EB300000F
:10A0900095B3000068A1000000000000000000006F
:10A0A000A5B30000ACB3000000000000DD1C000000
:10A0B00000000000BBB30000C2B3000070A10000AC
:10A0C0000000000000000000CAB30000D1B300008F
:10A0D00000000000811C000000000000EBB3000045
:10A0E000F3B3000000000000851B0000000000002A
:10A0F00008B400000FB4000000000000591B00006D
:10A10000000000001EB4000026B4000000000000A3
:10A110002D1B0000000000000000000000000000F7
:10A1200000000000000000000000000036B4000045
:10A130003BB40000000000007D7A00000000000039
:10A1400048B400004DB4000000000000757A000023
:10A1500000000000000000000000000000000000FF
:10A16000000000000000000000000000A0A00000AF
:10A17000000000002CA10000DCB40000E3B40000EB
:10A18000DCA100000000000000000000EC9B0000CB
:10A19000349C0000349C0000349C0000349C00007F
:10A1A0000EB50000F3B4000000000000891E00009E
:10A1B0000000000015B500001AB500000000000006
:10A1C0009D1D0000000000000000000000000000D5
:10A1D000000000000000000000000000000000007F
:10A1E000A0A100001CB6000023B6000020A20000C1
:10A1F0001D1F000000000000CCAB00005DB6000099
:10A2000000000000412100000201000000000000E9
:10A21000000000000000000000000000000000003E
:10A2200000000000F8A100003A000000E005002056
:10A23000000000003C0000201C000020D90C002081
:10A240001E000000DB840000349C00005C00002045
:10A25000552200008F7A0000AB7A0000D17A00000E
:10A26000BF7A000000000000D4B9000092B90000DD
:10A2700000000000E12E00000100000058BB0000BB
:10A280005EBB0000000000005D3500000100000022
:10A2900013BB00001BBB000000000000C134000025
:10A2A0000100000067BA00006EBA0000E4A20000DE
:10A2B00091350000010100002CBB000032BB000002
:10A2C000ECA2000000000000000000000000000000
:10A2D000FCA200000000000038A300000000000005
:10A2E00074A3000000000000B0A300000000000004
:10A2F000D8A30000000000003CA40000C5BC000082
:10A30000CFBC0000000000002D870000010000000D
:10A3100007BD00000EBD0000000000004F870000D8
:10A32000010000000000000000000000000000002C
:10A330000000000000000000FAB90000FCBD0000B1
:10A3400000000000938700000100000054AC0000F2
:10A3500014BE000000000000B587000001000000EE
:10A3600000000000000000000000000000000000ED
:10A3700000000000FAB90000AABD000000000000C3
:10A38000718700000100000054AC0000E9BD00002E
:10A3900000000000D787000001000000000000005E
:10A3A00000000000000000000000000000000000AD
:10A3B0006CBB000074BB0000000000008134000092
:10A3C000010000000000000000000000000000008C
:10A3D0000000000000000000B8BB0000C7BB000088
:10A3E000CCA20000000000000000000077BC0000CC
:10A3F0007EBC0000D4A200000000000000000000AD
:10A4000095BC00009ABC0000DCA2000005350000ED
:10A4100001010000ADBC0000B3BC0000F4A20000CC
:10A42000000000000000000000000000000000002C
:10A4300000000000000000000000000045BD00001A
:10A440004BBD0000000000000B8700000100000071
:10A4500079BD00007EBD000000000000A9340000AE
:10A4600001000000000000000000000000000000EB
:10A4700000000000000000000000002000000000BC
:10A4800000000B06020000008CA400000000000089
:10A4900082BE000024000207000000208ABE0000E7
:10A4A0001E000B1109BF00001BBF000008A5000023
:10A4B000CD440000000000006D4400008D8E0000BF
:10A4C000F58E000000000000038E00000000000078
:10A4D0000D440000F5450000A9440000158F000060
:10A4E00032BF000039BF000000000000CD44000072
:10A4F000010000000000000000000000000000005B
:10A50000000000000000000000000000E0A40000C7
:10A51000F1420000C142000000000000B548000008
:10A52000278F0000358F00004B8F0000578F0000F1
:10A53000638F000081470000758F0000000000005D
:10A54000FFFFFFFF000000500000000000000000BF
:10A55000002000406CA50000010000000600000083
:10A560000800010005000200070003005CA50000D0
:10A5700004000000E78F0000614C0000D98F00004C
:10A580000D4A0000C98F0000799100000D90000075
:10A59000399000006790000071900000AB900000BF
:10A5A000B7900000719000009B900000C3900000E5
:10A5B000D1900000ED900000DF900000E3900000DB
:10A5C00000200040020000000000000050A5000034
:10A5D000949B0000CC9B0000D49B0000E49B0000F7
:10A5E000EC9B0000F5FFFFFF5374617274696E67A6
:10A5F00020526164696F2054657374206578616DC1
:10A60000706C650A00556E61626C6520746F20671E
:10A6100065742074686520436C6F636B206D616E98
:10A62000616765720A00436C6F636B2072657175B8
:10A63000657374206661696C65643A2025640A005C
:10A64000436C6F636B20636F756C64206E6F742056
:10A65000626520737461727465643A2025640A002F
:10A66000436C6F636B2068617320737461727465EF
:10A67000640A004E52465F524144494F5F4D4F4479
:10A68000455F424C455F324D42495400446174611C
:10A6900020726174653A2025730A004E52465F525B
:10A6A0004144494F5F4D4F44455F424C455F314DFA
:10A6B000424954004E52465F524144494F5F4D4F0C
:10A6C00044455F4E52465F3235304B424954004E4E
:10A6D00052465F524144494F5F4D4F44455F4E5291
:10A6E000465F324D424954004E52465F5241444902
:10A6F0004F5F4D4F44455F4E52465F314D42495486
:10A7000000524144494F5F5458504F5745525F548F
:10A7100058504F5745525F4E6567343064426D0064
:10A72000545820706F7765723A2025730A005241A1
:10A7300044494F5F5458504F5745525F5458504FFB
:10A740005745525F4E6567333064426D0052414455
:10A75000494F5F5458504F5745525F5458504F57C8
:10A7600045525F4E6567323064426D005241444944
:10A770004F5F5458504F5745525F5458504F5745AC
:10A78000525F4E6567313664426D00524144494F15
:10A790005F5458504F5745525F5458504F57455289
:10A7A0005F4E6567313264426D00524144494F5FEC
:10A7B0005458504F5745525F5458504F5745525F69
:10A7C0004E65673864426D00524144494F5F5458AA
:10A7D000504F5745525F5458504F5745525F4E6542
:10A7E000673464426D00524144494F5F5458504FA2
:10A7F0005745525F5458504F5745525F3064426D31
:10A8000000524144494F5F5458504F5745525F548E
:10A8100058504F5745525F506F733364426D00522A
:10A820004144494F5F5458504F5745525F54585018
:10A830004F5745525F506F733464426D005452411C
:10A840004E534D49545F5041545445524E5F31313F
:10A85000303031313030005472616E736D69737312
:10A86000696F6E207061747465726E3A2025730A88
:10A87000005452414E534D49545F50415454455237
:10A880004E5F3131313130303030005452414E530F
:10A890004D49545F5041545445524E5F52414E44CD
:10A8A0004F4D00506172616D65746572733A0A00B4
:10A8B00044617461207261746520756E6B6E6F7790
:10A8C0006E206F7220646570726563617465643AAE
:10A8D0002025640A0D0A00545820706F7765722095
:10A8E000756E6B6E6F776E3A2025640A0054726144
:10A8F0006E736D697373696F6E20706174746572C5
:10A900006E20756E6B6E6F776E3A2025640A005369
:10A9100074617274204368616E6E656C3A202568BC
:10A9200068750A456E64204368616E6E656C3A20F6
:10A93000256868750A54696D65206F6E20656163CE
:10A9400068206368616E6E656C3A202575206D73B2
:10A950000A44757479206379636C653A2025752003
:10A9600070657263656E740A0A0025733A2062612D
:10A970006420706172616D657465727320636F75B8
:10A980006E740A004368616E6E656C206D75737439
:10A99000206265206265747765656E203020616E87
:10A9A000642038300A005374617274206368616EE9
:10A9B0006E656C2073657420746F3A2025640A00FC
:10A9C000456E64206368616E6E656C2073657420EB
:10A9D000746F3A2025640A0044656C6179207469BB
:10A9E0006D65206D7573742062652062657477658E
:10A9F000656E203020616E64203939206D730A0045
:10AA000044656C61792074696D6520736574207488
:10AA10006F3A2025640A005374617274207468656B
:10AA200020545820636172726965720A0025733A76
:10AA30002062616420706172616D6574657273205B
:10AA4000636F756E742E0A0053746172742074689B
:10AA500065206D6F64756C61746564205458206363
:10AA60006172726965720A00447574792063796352
:10AA70006C65206D757374206265206265747765FE
:10AA8000656E203120616E642039302E0A005258E4
:10AA90002073776565700A00545820737765657078
:10AAA0000A00546865206D6F64756C61746564207C
:10AAB0005458206861732066696E69736865640A1A
:10AAC000005265636569766564207061796C6F61B9
:10AAD000643A0A004E756D626572206F662070617F
:10AAE000636B6574733A2025640A00496E76616C65
:10AAF000696420444344432076616C75652070721C
:10AB00006F76696465640A0044434443207374614A
:10AB100074652025640A57726974652027312720DF
:10AB20006F722027302720746F20746F67676C6501
:10AB30000A00556B6E6F776E20617267756D656E7A
:10AB4000743A2025730A00556B6E6F776E20617220
:10AB500067756D656E743A2025732E0A00746F67F1
:10AB6000676C655F646364635F73746174650054EC
:10AB70006F67676C65204443444320737461746558
:10AB8000203C73746174653E2C20546F67676C655C
:10AB90002044432F444320737461746520726567B9
:10ABA0006172646C657373206F6620737461746581
:10ABB0002076616C7565007072696E745F727800E2
:10ABC0005072696E74205258207061796C6F6164A4
:10ABD0000073746172745F727800537461727420D0
:10ABE00052580073746172745F74785F737765652F
:10ABF00070005374617274205458207377656570C7
:10AC00000073746172745F72785F7377656570004A
:10AC100053746172742052582073776565700070A8
:10AC20006172616D65746572735F7072696E7400D4
:10AC30005072696E742063757272656E74206465FB
:10AC40006C61792C206368616E6E656C20616E6446
:10AC500020736F206F6E0073746172745F6475741B
:10AC6000795F6379636C655F6D6F64756C61746542
:10AC7000645F74780044757479206379636C65202F
:10AC8000696E2070657263656E74202874776F201A
:10AC9000646563696D616C206469676974732C20F5
:10ACA0006265747765656E20303120616E6420398D
:10ACB0003029203C647574795F6379636C653E006C
:10ACC0007472616E736D69745F7061747465726EB5
:10ACD0000053657420746865207472616E736D69C9
:10ACE0007373696F6E207061747465726E006F7536
:10ACF000747075745F706F776572004F75747075DE
:10AD00007420706F77657220736574203C73756270
:10AD10005F636D643E0073746172745F74785F6D1D
:10AD20006F64756C617465645F636172726965728A
:10AD300000537461727420746865206D6F64756C63
:10AD40006174656420545820636172726965720091
:10AD500073746172745F74785F6361727269657233
:10AD600000537461727420746865205458206361C4
:10AD7000727269657200646174615F72617465000A
:10AD800053657420646174612072617465203C7342
:10AD900075625F636D643E0063616E63656C004362
:10ADA000616E63656C2074686520737765657020DB
:10ADB0006F722074686520636172726965720074D5
:10ADC000696D655F6F6E5F6368616E6E656C005480
:10ADD000696D65206F6E2065616368206368616ED0
:10ADE0006E656C20696E206D7320286265747765CE
:10ADF000656E203120616E6420393929203C7469E8
:10AE00006D653E00656E645F6368616E6E656C00C3
:10AE1000456E64206368616E6E656C20666F72209B
:10AE20007468652073776565702028696E204D48C9
:10AE30007A20617320646966666572656E63652059
:10AE400066726F6D2032343030204D487A29203CB4
:10AE50006368616E6E656C3E0073746172745F63EB
:10AE600068616E6E656C0053746172742063686112
:10AE70006E6E656C20666F722074686520737765EE
:10AE80006570206F7220746865206368616E6E65FE
:10AE90006C20666F722074686520636F6E737461D6
:10AEA0006E7420636172726965722028696E204D2C
:10AEB000487A20617320646966666572656E6365B1
:10AEC0002066726F6D2032343030204D487A292050
:10AED0003C6368616E6E656C3E007061747465728F
:10AEE0006E5F72616E646F6D005365742074686587
:10AEF000207472616E736D697373696F6E20706117
:10AF0000747465726E20746F2072616E646F6D2E42
:10AF1000007061747465726E5F3131313130303080
:10AF2000300053657420746865207472616E736DAF
:10AF3000697373696F6E207061747465726E2074CA
:10AF40006F2031313131303030302E007061747407
:10AF500065726E5F3131303031313030005365749D
:10AF600020746865207472616E736D697373696FA4
:10AF70006E207061747465726E20746F2031303190
:10AF800030313031302E00706F733464426D0054B4
:10AF90005820706F7765723A202B342064426D0020
:10AFA000706F733364426D00545820706F77657210
:10AFB0003A202B332064426D00706F733064426D11
:10AFC00000545820706F7765723A20302064426DCB
:10AFD000006E65673464426D00545820706F776569
:10AFE000723A202D342064426D006E6567386442E9
:10AFF0006D00545820706F7765723A202D382064A8
:10B00000426D006E6567313264426D0054582070A5
:10B010006F7765723A202D31322064426D006E6583
:10B0200067313664426D00545820706F7765723A0C
:10B03000202D31362064426D006E656732306442E7
:10B040006D00545820706F7765723A202D32302091
:10B0500064426D006E6567333064426D0054582061
:10B06000706F7765723A202D33302064426D006E28
:10B070006567343064426D00545820706F77657294
:10B080003A202D34302064426D006E72665F314D7F
:10B090006269740031204D6269742F73204E6F72A3
:10B0A0006469632070726F7072696574617279206F
:10B0B000726164696F206D6F6465006E72665F32E5
:10B0C0004D6269740032204D6269742F73204E6F97
:10B0D000726469632070726F7072696574617279ED
:10B0E00020726164696F206D6F6465006E72665FC7
:10B0F0003235304B62697400323530206B626974CE
:10B100002F73204E6F726469632070726F70726962
:10B11000657461727920726164696F206D6F646516
:10B1200000626C655F314D6269740031204D626967
:10B13000742F7320426C7565746F6F7468204C6F48
:10B140007720456E6572677900626C655F324D628B
:10B1500069740032204D6269742F7320426C7565EA
:10B16000746F6F7468204C6F7720456E65726779D5
:10B1700000556E65787065637465642074657374DA
:10B1800020747970653A2025640A006E7266785FD3
:10B1900074696D65725F696E6974206661696C655A
:10B1A0006420776974683A2025640A00080420083E
:10B1B000044010000000000000000020286E696CB0
:10B1C00029004661696C656420746F207265626F46
:10B1D0006F743A207370696E6E696E6720656E6475
:10B1E0006C6573736C792E2E2E0A005A657068791F
:10B1F000722076657273696F6E2025642E25642E29
:10B2000025640A00557074696D653A202575206DB6
:10B21000730A005363686564756C65723A2025751E
:10B220002073696E6365206C6173742063616C6C5C
:10B230000A00546872656164733A0A002A004E413C
:10B24000002573257020252D3130730A00096F7099
:10B2500074696F6E733A20307825782C207072698B
:10B260006F726974793A2025642074696D656F7511
:10B27000743A20256C6C640A000973746174653A31
:10B280002025732C20656E7472793A2025700A008F
:10B29000556E61626C6520746F2064657465726DB3
:10B2A000696E6520756E7573656420737461636B78
:10B2B0002073697A6520282564290A0A00097374B5
:10B2C00061636B2073697A6520257A752C20756E11
:10B2D0007573656420257A752C2075736167652008
:10B2E000257A75202F20257A75202825752025257B
:10B2F000290A0A0025702049525120253032642045
:10B3000020202020287265616C2073697A652025D1
:10B310007A75293A09756E7573656420257A750901
:10B32000757361676520257A75202F20257A752031
:10B3300028257A75202525290A006379636C6573B1
:10B340003A202575206877206379636C65730A005D
:10B35000257020252D31307320287265616C207393
:10B36000697A6520257A75293A09756E7573656461
:10B3700020257A7509757361676520257A75202FF8
:10B3800020257A7520282575202525290A006B653A
:10B39000726E656C004B65726E656C20636F6D6DCF
:10B3A000616E6473006379636C6573004B65726EE4
:10B3B000656C206379636C65732E007265626F6FD4
:10B3C00074005265626F6F742E00737461636B73E7
:10B3D000004C6973742074687265616473207374BF
:10B3E00061636B2075736167652E007468726561B7
:10B3F0006473004C697374206B65726E656C2074A5
:10B400006872656164732E00757074696D65004BB8
:10B4100065726E656C20757074696D652E00766559
:10B420007273696F6E004B65726E656C2076657223
:10B4300073696F6E2E00636F6C6400436F6C6420E1
:10B440007265626F6F742E007761726D0057617262
:10B450006D207265626F6F742E005B25705D002039
:10B460002072657175697265733A2025730A0052FE
:10B47000454144590044495341424C4544006465A8
:10B4800076696365733A0A002D202573002028250C
:10B4900073290A002D2025730A00505245204B4580
:10B4A000524E454C20313A0A002D204E6F6E650AEF
:10B4B00000505245204B45524E454C20323A0A002E
:10B4C000504F53545F4B45524E454C3A0A00415041
:10B4D000504C49434154494F4E3A0A0064657669DD
:10B4E00063650044657669636520636F6D6D616EA9
:10B4F0006473004C69737420636F6E66696775725C
:10B5000065642064657669636573206279206C6583
:10B5100076656C73006C697374004C697374206396
:10B520006F6E6669677572656420646576696365C8
:10B5300073005573696E6720646174612077696474
:10B5400074682025640A00496E636F7272656374C3
:10B5500020646174612077696474680A00526561CF
:10B56000642076616C756520307825780A00577202
:10B570006974696E672076616C756520307825780E
:10B580000A006465766D656D206C6F61642073756B
:10B5900070706F7274732073657474696E67206263
:10B5A0007970617373206F6E20612073696E676CB0
:10B5B0006520696E7374616E63652E0A004C6F615D
:10B5C00064696E672E2E2E0A707265737320637421
:10B5D000726C2D78206374726C2D7120746F2065ED
:10B5E00073636170650A004E756D626572206F66E7
:10B5F00020627974657320726561643A2025640A5B
:10B60000002D2D002D6500556E6B6E6F776E206FCF
:10B610007074696F6E20222573220A006465766D4E
:10B62000656D00526561642F77726974652070687A
:10B6300079736963616C206D656D6F7279226465E1
:10B64000766D656D2061646472657373205B7769E4
:10B65000647468205B76616C75655D5D005573612F
:10B6600067653A0A6465766D656D206C6F6164206C
:10B670005B6F7074696F6E735D205B61646472658B
:10B6800073735D0A4F7074696F6E733A0A2D6509A2
:10B690006C6974746C652D656E6469616E2070618F
:10B6A00072736500756172743A7E24200073686558
:10B6B0006C6C5F7561727400537562636F6D6D6160
:10B6C0006E64733A0A006E6F74207465726D696EF1
:10B6D000617465643A2025630A00506C6561736586
:10B6E0002073706563696679206120737562636F8A
:10B6F0006D6D616E642E0A004572726F723A20722F
:10B700006571756573746564206D756C7469706CB2
:10B71000652066756E6374696F6E20657865637504
:10B7200074696F6E730A003A20636F6D6D616E64A9
:10B73000206E6F7420666F756E6400546F6F206D9D
:10B74000616E7920617267756D656E747320696EC4
:10B750002074686520636F6D6D616E642E0A00252C
:10B76000733A2077726F6E6720706172616D6574D5
:10B77000657220636F756E740A005741524E494ED0
:10B78000473A2041207072696E7420726571756548
:10B7900073742077617320646574656374656420D5
:10B7A0006F6E206E6F7420616374697665207368B4
:10B7B000656C6C206261636B656E642E0A000A25FD
:10B7C000732573005368656C6C20746872656164DE
:10B7D000206572726F723A20256400506C65617347
:10B7E0006520707265737320746865203C546162D3
:10B7F0003E20627574746F6E20746F2073656520CF
:10B80000616C6C20617661696C61626C6520636F4C
:10B810006D6D616E64732E0A00596F752063616EE1
:10B8200020616C736F2075736520746865203C54CB
:10B8300061623E20627574746F6E20746F20707246
:10B840006F6D7074206F72206175746F2D636F6DF2
:10B85000706C65746520616C6C20636F6D6D616EDA
:10B860006473206F722069747320737562636F6DE7
:10B870006D616E64732E0A00596F752063616E20CE
:10B8800074727920746F2063616C6C20636F6D6DCE
:10B89000616E64732077697468203C2D683E206F68
:10B8A00072203C2D2D68656C703E20706172616D58
:10B8B0006574657220666F72206D6F726520696EA7
:10B8C000666F726D6174696F6E2E0A000A53686547
:10B8D0006C6C20737570706F72747320666F6C6C13
:10B8E0006F77696E67206D6574612D6B6579733A4A
:10B8F0000A20204374726C202B202861206B65790C
:10B900002066726F6D3A206162636465666B6C6E6F
:10B91000707577290A2020416C7420202B20286123
:10B92000206B65792066726F6D3A206266290A5035
:10B930006C6561736520726566657220746F207333
:10B9400068656C6C20646F63756D656E7461746995
:10B950006F6E20666F72206D6F7265206465746112
:10B96000696C732E0A000A417661696C61626C65CC
:10B9700020636F6D6D616E64733A0A00253038582C
:10B980003A2000253032782000202020007C007CE6
:10B990000A005072696E7473207468652068656C63
:10B9A00070206D6573736167652E001B5B256425D0
:10B9B00063001B5B313B3325646D001B5B3430330C
:10B9C00025646D002573252D2A730025733A002DFB
:10B9D00068002D2D68656C7000202D20002020004F
:10B9E0004C6F7374206C6F67733A20256C750A0076
:10B9F0005B2533645D2025730A006F66660025733E
:10BA00003A257325730A0020756E6B6E6F776E2072
:10BA1000706172616D657465723A20004563686F8C
:10BA2000207374617475733A2025730A004E6F2079
:10BA3000726573706F6E73652066726F6D207468C7
:10BA400065207465726D696E616C2C20617373750D
:10BA50006D65642038307832342073637265656EAA
:10BA60002073697A650A00726573697A6500436FAD
:10BA70006E736F6C652067657473207465726D6991
:10BA80006E616C2073637265656E2073697A6520E0
:10BA90006F7220617373756D65732064656661757F
:10BAA0006C7420696E206361736520746865207210
:10BAB0006561646F7574206661696C732E204974CA
:10BAC000206D757374206265206578656375746593
:10BAD00064206166746572206561636820746572B4
:10BAE0006D696E616C207769647468206368616E4B
:10BAF000676520746F20656E7375726520636F7261
:10BB000072656374207465787420646973706C6105
:10BB1000792E00686973746F727900436F6D6D617F
:10BB20006E6420686973746F72792E007368656C37
:10BB30006C0055736566756C2C206E6F7420556EA5
:10BB400069782D6C696B65207368656C6C20636F18
:10BB50006D6D616E64732E00636C65617200436C81
:10BB60006561722073637265656E2E00646566613F
:10BB7000756C7400417373756D652038302063688F
:10BB80006172732073637265656E2077696474688F
:10BB900020616E642073656E64207468697320731D
:10BBA000657474696E6720746F20746865207465AD
:10BBB000726D696E616C2E006261636B737061639C
:10BBC000655F6D6F646500546F67676C65206261C7
:10BBD000636B7370616365206B6579206D6F64655D
:10BBE0002E0A536F6D65207465726D696E616C739A
:10BBF00020617265206E6F742073656E64696E6774
:10BC0000207365706172617465206573636170652E
:10BC100020636F646520666F72206261636B73706E
:10BC200061636520616E642064656C657465206283
:10BC30007574746F6E2E205468697320636F6D6D18
:10BC4000616E6420666F72636573207368656C6CE7
:10BC500020746F20696E74657270726574206465FB
:10BC60006C657465206B6579206173206261636B1C
:10BC700073706163652E00636F6C6F727300546F35
:10BC800067676C6520636F6C6F7265642073796E93
:10BC90007461782E006563686F00546F67676C6528
:10BCA000207368656C6C206563686F2E0073746127
:10BCB0007473005368656C6C207374617469737479
:10BCC0006963732E006261636B7370616365005317
:10BCD000657420646966666572656E742065736359
:10BCE00061706520636F646520666F7220626163B6
:10BCF0006B737061636520616E642064656C65744C
:10BD000065206B65792E0064656C6574650053650C
:10BD100074207468652073616D652065736361705C
:10BD20006520636F646520666F72206261636B7368
:10BD30007061636520616E642064656C6574652064
:10BD40006B65792E00726573657400526573657456
:10BD5000207368656C6C20737461746973746963B3
:10BD60007320666F7220746865204C6F6767657218
:10BD7000206D6F64756C652E0073686F7700476582
:10BD800074207368656C6C20737461746973746972
:10BD9000637320666F7220746865204C6F676765F7
:10BDA00072206D6F64756C652E0044697361626CFE
:10BDB00065207368656C6C206563686F2E20456430
:10BDC0006974696E67206B65797320616E64206D9C
:10BDD0006574612D6B65797320617265206E6F7477
:10BDE0002068616E646C656400456E61626C6520FC
:10BDF0007368656C6C206563686F2E0044697361BD
:10BE0000626C6520636F6C6F7265642073796E7409
:10BE100061782E00456E61626C6520636F6C6F7295
:10BE200065642073796E7461782E001B5B366E003A
:10BE3000436F6D6D616E6420627566666572206920
:10BE40007320746F6F2073686F727420746F206535
:10BE50007870616E6420616C6C20636F6D6D616ED3
:10BE60006473206D61746368696E672077696C64C0
:10BE700063617264207061747465726E3A20257318
:10BE80000A00464C4153485F30005352414D5F30E9
:10BE9000006E6F742000484620636C6F636B3A0A33
:10BEA00000092D20257372756E6E696E67202875E6
:10BEB000736572733A202575290A00092D206C617B
:10BEC00073742073746172743A202575206D732029
:10BED000282575206D732061676F290A00092D20C0
:10BEE0006C6173742073746F703A202575206D73C4
:10BEF00020282575206D732061676F290A004C4644
:10BF000020636C6F636B3A0A006E72665F636C6FDE
:10BF1000636B5F636F6E74726F6C00436C6F636B07
:10BF200020636F6E74726F6C20636F6D6D616E64F1
:10BF30007300737461747573005374617475730066
:10BF4000434C4F434B004750494F5F3000554152DF
:10BF5000545F3000000001010100000001010000F9
:10BF600000000101000000005465726D696E616C93
:10BF700000525454005345474745520069646C656C
:10BF8000006D61696E00756E6B6E6F776E00706527
:10BF90006E64696E670070726573746172740064B8
:10BFA0006561640073757370656E646564006475C3
:10BFB0006D6D790061626F7274696E67007175658D
:10BFC0007565640076332E302E39392D6E637331EA
:10BFD000002A2A2A20426F6F74696E67205A6570A2
:10BFE000687972204F53206275696C642025732034
:10BFF0002573202A2A2A0A00737973776F726B716E
:04C00000000000003C
:10C0040000030000500000000A000000320000009D
:10C01400B773000050A200002CA20000282D0020BD
:10C02400000000000000000000000000000000000C
:10C03400000000000000000040000000202D00204F
:10C0440000000000000000000000000000000000EC
:10C0540000000000000000000800000000000000D4
:10C064000100000074000020000000000000000037
:10C0740000000000202B0020000000000000000051
:10C0840000000000000000000000000000000000AC
:10C0940000020000FFFFFFFFBF8D00000000000052
:10C0A40000000000F90C0020200000000000000047
:10C0B4000000000000C20100000103009C000020F9
:10C0C40000000000000000000090D0030000000009
:10C0D400000000000000000000000000000000005C
:10C0E400000000000000000000000000000000004C
:10C0F400000000000000000000000000000000003C
:10C10400000000000000000000000000000000002B
:10C11400000000000000000000000000FF0000001C
:10C124000000000000000000FFFF0F002C010020B1
:0CC134002C010020340100203401002008
:10C14000515600007D94000000000000078A0000A6
:10C150001C9C0000F991000000000000078A00000C
:10C1600000000000078A000000000000078A0000AD
:10C17000A95B00007D94000000000000078A000019
:10C1800000000000D55D000000000000078A0000EC
:10C1900000000000078A000000000000078A00007D
:10C1A00000000000078A000000000000078A00006D
:10C1B00000000000078A000000000000078A00005D
:10C1C00000000000078A0000000000002550000069
:10C1D00000000000078A000000000000078A00003D
:10C1E00000000000078A000000000000078A00002D
:10C1F00000000000078A000000000000078A00001D
:10C2000000000000078A000000000000078A00000C
:10C2100000000000078A000000000000078A0000FC
:10C2200000000000078A000000000000078A0000EC
:10C2300000000000078A000000000000078A0000DC
:10C2400000000000078A000000000000078A0000CC
:10C2500000000000078A000000000000078A0000BC
:10C2600000000000078A000000000000078A0000AC
:08C2700000000000078A000035
:0CC27800000000000000000000000000BA
:0400000300003F6D4D
:00000001FF
